S0140000755461736B65725F56312E342E73726563E9
S10B0000FC2F0020813F0000E9
S11304000000000000000000FFFFFFFFBE03FFFF2D
S1130410F8B50C1C131E022B4ED0042A02D0002A5D
S11304200BD039E000780324822848D125490D22D5
S11304300878254905F042FD41E006788022311C08
S1130440914321293AD1C1798279204D0F02174372
S113045076B22F80002E31DA2B804378FE2B02D027
S1130460FF2B2BD114E08578002D27D1C778002FDE
S113047024D10679002E21D1407900281ED1012AE9
S11304801CD100291AD112490878124905F016FD29
S1130490082C11D9083CA4B20C4B1A88002A0BD0A2
S11304A00D4F00253D70944202D31D80032406E0C5
S11304B0161B1E80062402E0002400E00424201CF5
S11304C0F8BDC04604F1FF1FC0F0FF1FF6F0FF1F88
S11304D028F3FF1F899C0000F4F0FF1FF8B51B4DA3
S11304E0002128780A1C05F0E9FC041C184E336826
S11304F0002B22D01748844219D9174F0020011C21
S11305003A6809F05DFA00280DD1144980230A687D
S1130510287851699A0005F0D1FC396810480131F6
S11305202418A4B239603768013F3760DEE72878C1
S113053040210C4A05F03CFA06E00C2CF7D9287847
S113054009490D2205F0BAFCF8BDC04604F1FF1FAD
S11305500CF1FF1FFF010000FCF0FF1F24F1FF1F3F
S113056000FEFFFF75100000C0F0FF1F38B5304BD0
S1130570041C1A680725002A58D12E48211C04227D
S113058005F052FD0425002850D1607B00284DD190
S1130590A17B01390F2949D8257BE37B7F2D16D90F
S11305A0232B1ED006D8122B3FD01A2B09D0032B95
S11305B025D13AE0282B14D0A82B12D0252B1ED1FC
S11305C033E0201C0F304278510929D017E01E2B4C
S11305D02BD002D8002B28D011E02A2B01D0AA2B33
S11305E00DD11548882302680725118B19421DD1A6
S11305F0124DF02002223A212870AA702973104D5E
S1130600211D281D042205F09BFB281C211C0830F9
S113061008310422012405F093FB2C73042505E022
S113062085783F232B403F2BE9D10725281C38BD73
S1130630F8F0FF1FD39B000024F1FF1F10F1FF1FF0
S1130640C0F0FF1FF0B5C34B0330C07F1A78AFB0C2
S11306500190002A59D1C04904260D681F35281C71
S113066005F010FD440001D0A61CF6B2BB4F38685B
S1130670002806D1301C03F0EFFF03233860067016
S113068043703968002C02D18C70CC7008E02A7851
S11306900231002A04D000240A7001354C70F6E7B8
S11306A009AA0027AE4E0320012550747524391C75
S11306B0052097735581D780978015749474099693
S11306C005F028FAA34B0EAA187002218023917317
S11306D0A44ED90080209474D5738400D180402521
S11306E0391C05209581948014810E9605F012FA28
S11306F09D4A1070381C09F087F99C4F386004E05B
S1130700E07801280AD0752829D00EAC0198211C64
S1130710052205F063F90028F2D151E02479CB2CAD
S113072018D007D8CA2CF0D10220002104F02AFBEB
S11307308F4825E0CC2C04D0DD2CE6D1FFF7CEFE8B
S1130740E3E78C488C4A8D4E0023036013603360CA
S11307508B4815E0002104F015FB8A4810E0694637
S1130760227901983D3105F039F96579FE2DCCD116
S1130770854805F0C3FBA079012105F0D0FB83482F
S113078005F0BCFBC1E77B4E28783768002F30D0DA
S11307907A4F7F493B6880229200C918D31A9AB2D3
S11307A005F01CF931683B680A1A7A49C0183260AE
S11307B0386088420BDC6F4F3968002900D11BE197
S11307C0694D287805F01AF90028DCD120E1724B34
S11307D06F491A68501C1860002009F003F9366844
S11307E000223A60002EE6D07520042103F048FE72
S11307F00EE1211C802205F0F1F8684E0FA90422B5
S1130800301D05F09DFA2878012137727772B7728E
S1130810F772377305F004F9E07B032804D06048CD
S11308206049122205F08CFA217BE37B7F2900D8F2
S113083086E0232B5ED00AD8122B24D01A2B27D083
S1130840032B00D0D8E0287855491222DDE0282B6C
S11308502FD0A82B2DD0252B00D0CDE0434B04A9BD
S11308601F6800260E714E713A8D3E69100ACA71D6
S1130870330E320A370C88718A700B704F70CE7049
S113088028780822C1E0277C780900D1BAE0B1E0D9
S113089003AE0422301C444905F052FA334802687E
S11308A0138BD90601D58021B1702878311C04221C
S11308B0ABE0657CA07C277D06042906E27C3143FD
S11308C0394315023448294301602B4EA77DE17D4D
S11308D0A82B09D1627D38041506277E28433843A6
S11308E00B02011C194301E03B0219433160FFF77D
S11308F0F5FD65E7A67DE17D370206AE0C220F43C8
S1130900301C2A4905F01CFA184A88211068038B08
S11309100B420DD0990601D5022200E001220069A4
S11309203272030A010C020EF071B37171713271EB
S113093028783B1C0C2F00D90C239AB2311C64E09C
S11309402A2B35D0AA2B33D0002B55D1227C570922
S113095052D04FE028F3FF1F74F4FF1F00F1FF1F74
S1130960110400006D05000004F1FF1F24F1FF1FB6
S11309702E9C0000F8F0FF1F0CF1FF1F08F1FF1F71
S1130980129C00001E9C00003B9C0000489C000040
S113099028F1FF1FFF010000FCF0FF1FC0F0FF1F44
S11309A010F1FF1FF09B0000719C0000759C00007B
S11309B0657CA07C227D01042E06E77C0E43164351
S11309C03D0214482E430660A27D134EE17DAA2BFE
S11309D009D1677D10043D06227E284310430B0293
S11309E0011C194301E013021943316031684F02BD
S11309F03760E5E601223273287808490D2205F0B4
S1130A005DFADDE628780649242205F057FAF3E773
S1130A102FB0F0BDFCF0FF1FF8F0FF1FC0F0FF1F68
S1130A204D9C000012230380004870478A9C0000FC
S1130A302023038000487047A99B000000B50528C7
S1130A400DD8084B8200D3581A78002A05D1131CFC
S1130A50032805D1044803681A780A8000E00023BB
S1130A60181C00BDD89B000000F1FF1F00B50B78D7
S1130A700278002B05D0013001319A42F7D00020D2
S1130A8007E0202A04D80178202902D10130FAE7AE
S1130A90181C00BD30B50368021C1978202904D144
S1130AA01568013301351560F7E71D1D0020AB42C1
S1130AB013D019782F2910D90C1C303C0001E4B252
S1130AC080B20133092C01D93739CCB20F210C4043
S1130AD02043146801341460E9E730BD00B50368AD
S1130AE01A78202A06D01978002903D0202901D0A9
S1130AF00133F8E71A78202A01D10133FAE70360B9
S1130B0018784342584100BD30B50023DC006442EC
S1130B10183493420AD0051CE540ECB2251C203D54
S1130B205A2D00D92E24CC540133EFE7C81830BD18
S1130B3008B5054805F0E2F9044805F0DFF9044872
S1130B4005F0DCF908BDC04690A20000A09B00009F
S1130B50D0A2000008B5044805F0D0F9034B18688A
S1130B60373005F0CBF908BDA2A2000078F4FF1FCE
S1130B7010B50C1C05F0C2F9084805F0BFF9084B84
S1130B801868018C0C4004D0064805F0B7F9012020
S1130B9003E0054805F0B2F9201C10BD29BB000094
S1130BA078F4FF1FBAA20000C4A20000F0B52C4ADA
S1130BB0071C13780C2043432A4E8BB0F1180D798F
S1130BC003A801951B224D7920219C5905F0AFF80B
S1130BD0002F04D0BD4225DD0C34013DFAE7224844
S1130BE005F08CF91E4F0C223B785343F618B0687D
S1130BF005F084F91D4805F081F913E0206805F03B
S1130C007DF9019B011C387899421EDB03A901225E
S1130C1005F054F9606805F071F9154805F06EF9AE
S1130C200C34013D002D15D0124F0021387842229A
S1130C3005F044F90028E1D1387840210E4A04F047
S1130C40B7FE0E480560012007E0019A561AB2B2B9
S1130C5003A9DDE7094C281C25600BB0F0BDC04694
S1130C6057F4FF1F0CA20000CFA20000D3A2000083
S1130C70D0A20000E6F0FF1F6D1000002CF3FF1F50
S1130C8008B5094B187808280AD108490A68002AC7
S1130C9004D01068002801D005F030F9044800E0C1
S1130CA0044805F02BF908BD57F4FF1F30F3FF1F6C
S1130CB077AE0000BDA7000008B5084B984205D9DF
S1130CC04008002105F02BF9054804E0400200210A
S1130CD005F025F9034805F011F908BDFFFF7F0071
S1130CE0EBA20000F3A20000F0B5BC4CA5440191B6
S1130CF0041E092C00D10AE2112800D181E308283E
S1130D0000D157E1152800D1B8E11D2800D178E3BE
S1130D101E2800D175E30B2800D197E2B04D286856
S1130D20002803D1642107F06FFF2860296802239B
S1130D300E8F1E4009D1301C07F08AFF002801D015
S1130D40A8485CE3A849286808601C2C00D958E32B
S1130D50201C08F06BFE1D00720209020002BF0095
S1130D60BF00560333022F01DC01DC017B021402B5
S1130D7056035603560356035603560356035603A7
S1130D80930140021D005603AE0056035603AE0005
S1130D90964F3E68002E07D10198934908F040F918
S1130DA0002801DA92482AE3924E012114A88F22E6
S1130DB0B18130603281172C01D0002300E002237E
S1130DC039683375002919D18B4805F097F82868DC
S1130DD0006805F093F82A68D38E032B02D987485C
S1130DE005F08CF80198002804D00178002901D07E
S1130DF005F084F8824805F081F801E000253D60A3
S1130E00804D00212878922205F058F800280AD154
S1130E10287840217C4A04F0CBFD0420172C00D113
S1130E20B1E00120AFE07048311C07F071FD009083
S1130E307089002809D0172C02D1744805F05EF897
S1130E402878728914A905F039F8009A0F32D7D19D
S1130E500021708A05F063F86D4805F04FF8002111
S1130E60706805F05CF86B4805F048F80021308A9A
S1130E7005F055F8684805F041F800211822301CA7
S1130E8004F055FF002008F0BFFD048B610709D56D
S1130E90066B721C06D02B3000787043FFF70CFFF2
S1130EA05E48ACE203236D2100203B6008F05CFD4A
S1130EB06AE01C2C01D15A4B00E05A4B2A68019875
S1130EC003A908F0D1FB002802DA574805F016F808
S1130ED003A86CE0554E6D22311C3F310A70042C7E
S1130EE001D0112300E0524B404F3868022802D150
S1130EF0042C39D108E02A680198311C08F0B4FBAD
S1130F00022800D078E1F3E74A4C8022217852008D
S1130F1014A804F00CFF277880230137301C14A98F
S1130F205A00277008F01CF9051E01D042482EE033
S1130F30424804F0E3FFB068291C04F0F0FF32E0FB
S1130F4080220025301C14A952003D6007F0C4FF24
S1130F5000281BD1B28F90421CDB207814A904F026
S1130F60ADFFB48FFF2C1ED9264C8023207800219E
S1130F705A0004F0A3FF0028E2D120784021224A3D
S1130F8004F016FD0220386001203BE22C4804F0F6
S1130F90B5FF08E014A90B5C0A3B702B01D92E2580
S1130FA00D540130D7E7274804F0A8FF301C08F09F
S1130FB095F826E2019804F081FE071C224804F00B
S1130FC09DFF381C842104F0A1FF002014A93A1CC1
S1130FD008F0F6FC00283BD01C4810E2ACFDFFFFF3
S1130FE030F3FF1FFAA2000040F3FF1F70F4FF1F4D
S1130FF00DA3000058F4FF1F21A30000FFBB000055
S11310002CA30000E6F0FF1F6D10000030A30000C9
S113101034A3000041A300004AA3000059A3000028
S113102001C000000140000061A3000070F3FF1F35
S113103012080000CDF0FF1F7CA3000089A300006C
S11310409CA30000ACB90000C2A30000D2A300001E
S1131050874C14AD201C04F051FF94AE271C0024CF
S113106028599421043404F051FF402CF8D1381C41
S1131070403504F043FFB542F1D1C2E1019804F0D8
S11310801DFE051C01A8FFF729FD0022904203D193
S1131090019804F013FEC2B20023D1188024C8B210
S11310A014AFA600B34202D0F8540133F5E77148F7
S11310B004F024FF281C842104F028FF6E4A8023B6
S11310C09905116001A8FFF709FD002801D0012648
S11310D005E0019804F0F2FDC6B2002EF7D02C1CF6
S11310E00020391C221C08F07DFC002801D0634834
S11310F000E0634804F002FF01347019C2B2E3B2A5
S11311009A42EDD180255C49AF050F6079E15D48D5
S113111004F0F4FE01985C49032204F085FF0028E2
S113112007D15A4804F0EAFE0198022204300190E3
S113113003E0574804F0E2FE00220A2C01D1012406
S113114022430020019908F08DFB002801D051486A
S113115055E1514853E12968019808F043FB002800
S113116000D14EE14D484AE12A68019803A94C4B4D
S113117008F07AFA022800D143E14A483FE1019F8E
S11311803C787E1C202C04D0371C002CF8D1464817
S113119035E1002038702A68019803A9231C08F05F
S11311A063FA002801DA414829E1301C03A907F059
S11311B04BFF002800D124E13D4820E12968019833
S11311C008F0B4FA411C01D13A4818E1002800D1D2
S11311D017E1394813E1019804F089FD071C0198CF
S11311E0027801300190202AF9D12A6803A9022348
S11311F008F03AFA022801D0304800E1002008F053
S113120003FC391C056B041C002203A808F004F934
S113121003A808F05FFB00280DD1294804F06EFEF6
S1131220266B701B05D0102104F079FE254804F0CC
S113123065FE0F48E3E02448E1E02968019808F0DE
S11312409DF8002800D1DCE02048D8E0002008F018
S1131250DBFB041C1E4804F051FE218B802252004B
S11312600A4001D01B48CAE08D0637D41A4846E02C
S1131270ACB90000DEA300000CF10F40F1A30000A4
S113128008A4000010A400001FA4000023A4000070
S113129027A400002BA400003AA4000059A40000D5
S11312A0020600006BA4000080A4000093A40000C8
S11312B09FA40000AFA40000BFA40000B1A30000DD
S11312C0CFA40000EBA40000FBA400000FA50000C5
S11312D01EA5000029A5000038A50000131CE6186F
S11312E0493637785020C1186D464F550133202FA9
S11312F000D01A1C0B2BF2D1002314A8835404F041
S1131300FDFD424804F0FAFD2069FFF7D5FC404892
S113131004F0F4FD268B710602D53E4804F0EEFD80
S1131320278BFA0602D53C4804F0E8FD3B4D281C07
S113133004F0E4FD208B2E1C850652D5384804F0B9
S1131340DDFD1821208D04F0EAFD364804F0D6FDB9
S1131350211C2B310A78208D1821504304F0DFFD25
S1131360314804F0CBFD9C21606804F0CFFD2F4888
S113137004F0C4FD9C21206A04F0C8FD2C4804F04C
S1131380BDFD9C21E06904F0C1FD2A4804F0B6FDCE
S1131390231C2A331878182104F0C1FD264804F0D0
S11313A0ADFD9C21A06804F0B1FD244804F0A6FD25
S11313B09C21606A04F0AAFD214804F09FFD9C2151
S11313C0E06A04F0A3FD1F4804F098FD9C21206B03
S11313D004F09CFD1C4804F091FD606B9C2104F01A
S11313E095FD1A4804F08AFD0027E5193835287858
S11313F09121013704F08AFD102FF6D1301C04F03E
S11314007DFD00209527BF00BD44F0BD0FA700005F
S1131410BAAC000046A500004CA50000ACB9000021
S11314205DA500006FA500007DA500008DA500004E
S113143098A50000A2A50000B2A50000B7A5000071
S1131440C7A50000D2A50000E1A50000ECA500009E
S113145038B5051C0C1C0E48291C04F0F2FD0028AC
S113146010D00C48291C04F0ECFD002804D00A48D4
S113147004F044FD01200AE0084B19680A8CA243D9
S11314800A8404E0054D2B68198C0C431C8438BD78
S1131490F1A50000F8A5000000A6000078F4FF1FE5
S11314A030B50330C57F8BB002AC281C211C05224B
S11314B004F094FA002855D0E3782279012B02D065
S11314C0412B4AD133E0DD2A18D127480468002C87
S11314D00DD0012C02D10020011C06E01720042CA1
S11314E002D0022C03D105200021FFF7FDFB1F4A87
S11314F010680028D8D0FFF759FBD5E7BF2AD3D10D
S1131500194C2268032ACFD1002008F07DFA016B20
S11315104A1C09D02B3000784843FFF7CDFB144810
S113152004F0ECFCFFF7ACFB00232360BCE7281CB1
S1131530211C04F053FA2078042808D1684669462F
S113154007300931012204F0FBFB0A4802E00328BA
S1131550AAD1094804F0D2FCA6E7281C211C04F0F7
S11315603DFAA1E70BB030BD70F4FF1F2CF3FF1F51
S113157059A3000013A6000024A6000008B50A1C05
S11315800349031C0878191C04F098FC08BDC046E4
S113159084FBFF1F10B5174B174A1B681268988B02
S11315A09188012488420BD1181C4C300088918EFC
S11315B0884205D1DC1C917AE07F441A611E8C417B
S11315C012891B8C28205340034201D002210C4372
S11315D00422134200D01443DA0601D508231C4325
S11315E0012001F03DFBE30702D5042001F0B6FB26
S11315F010BDC04678F4FF1F74F4FF1F38B5051CF6
S1131600164C022817D021681822154803F098F8C0
S11316102168144818313C2203F092F8012D1BD0A4
S1131620022003F0C6F821680F4818313C220068F4
S113163004F086FB10E00C4B20681968038C0A89BF
S113164053402B4201D0012007E00849182204F03E
S1131650EBFC0028D7D0F6E7002038BD78F4FF1F54
S1131660048000001C80000074F4FF1F9DFBFF1F1A
S113167010B5084C206801F08BFA20680649062250
S1131680023004F05DFB206804493C22183004F069
S113169057FB10BD78F4FF1F87FBFF1F50B30000FA
S11316A0F8B5204B051C1421186808F0C9F91E4927
S11316B0061C08F0C5F92A1C0021041C04F04AFA8F
S11316C0612773232022442179250371027041701C
S11316D08770C5704271871D13484443351BE1264A
S11316E03101281C08F0ACF93A1C0021041C04F058
S11316F031FAE12211014C433A262C1B0670471C97
S11317003C21201C08F09CF93A1C0221051C04F021
S113171021FA3C235D430670421C0221601B04F045
S113172019FAF8BDBCFBFF1F8051010038B50E4B00
S1131730021C1B689C78D8782502401984B29D79D4
S11317405879D97900041B792D022D1869181806C7
S11317500818022104F0FEF92D2202700A21421C0D
S1131760201C04F0F7F938BD78F4FF1F7FB5054855
S113177004F0C4FB01A8FFF7D9FF01A804F0BEFBE5
S113178007B000BD3EA60000802310B55900884272
S11317900BD1134B0224198800291FD1114A138835
S11317A0002B1BD101F02AFA03E080220D4C90009B
S11317B020800D48802104884A00944202D12020D0
S11317C001F01CFAFFF7D2FF0024FFF7B1F9FFF78D
S11317D0C1F9064B201C1C70FFF7E8F9201C10BD52
S11317E054F4FF1F34F3FF1F3CF3FF1F57F4FF1F94
S11317F000B532280ED0332818D0312823D1134B0A
S1131800134A186812681968124B10401B688B43FE
S1131810184316E00D490E4A0E4B08681268096811
S11318201B6810408B43184380000AE00A490B4AA6
S11318300B4B0868126809681B6810408B431843F7
S11318408006C00F00E0002000BDC04614F10F4028
S113185000F10F4010F10F40D4F00F40C0F00F40E2
S1131860D0F00F40F7B5144E0125336800241A1C3C
S11318704E32107850330090198831200191471C62
S1131880FFB2FFF7B5FF002800D02C436D00EDB286
S1131890381E3928F3D1FFF77DFE36686A46107882
S11318A09188331C4E335036187031805C700020A0
S11318B0FFF7A4FEF7BDC04678F4FF1F00B5322839
S11318C008D033280AD031280ED1084B1868C143F8
S11318D0C80F0AE005480268510F02E0044A136881
S11318E059090120884300E0002000BD14F10F4095
S11318F0D4F00F4038B5051C303D0020032D72D8BC
S1131900281C08F089F8020905078020040605E070
S1131910202403E0002401E08024A405EDB264291E
S11319200AD002D8612904D15CE0692904D06F2966
S11319302DD00121484256E0012D10D0002D0ED0AB
S1131940022D1BD128488022016853010B430360F8
S11319500320021C211C02F0CBFB24480BE0224B89
S113196080221968900108431860211C0420032276
S113197002F0BEFB1E480368A34303601D4C012212
S11319802168AA404E310878904308702AE0012D5E
S113199010D0002D0ED0022D1BD1134B80221868BD
S11319A05101014319600320211C042202F0A0FB11
S11319B00E4B0BE00C488022016893010B4303603B
S11319C00420211C021C02F093FB094B18680443F9
S11319D01C60084C01222168AA404E310B78151C6A
S11319E01D430D70002038BD38800440D4F00F40F2
S11319F014F10F4078F4FF1F00B5002905D0144BF3
S1131A00C022196892010A431A60124BC10704D517
S1131A101968802212060A4302E019684A00520833
S1131A201A601968820703D5802292050A4301E0EF
S1131A30094A0A401A60094B2022410702D5196855
S1131A400A4302E018689043021C1A6000BDC046B5
S1131A503880044000F10F40FFFFFFDFC0F00F406B
S1131A60F8B5B04D01212B6801241A1C4E324F33B6
S1131A701778187838401870FFF7BEFF30206921B6
S1131A80274200D06F21461C6400F6B2FFF732FFF4
S1131A90E4B2382E01D0301CF1E76120411C6238D9
S1131AA0CFB20E2809D807F0B7FF111A23323942F2
S1131AB04B545D666F92927881009B4E802233680E
S1131AC05101194380243160660019E0964B80214E
S1131AD01E684C01344380221C60960010E0924E34
S1131AE08024316862010A4380203260C60007E026
S1131AF08D4E8022346850012043802330601E01C3
S1131B000320311C042202F0F3FA88485CE0864882
S1131B10802103684E0133430360F1E7824B802642
S1131B20196874010C4380221C609601E8E77E4B1F
S1131B3080241E686201324380201A60C601DFE7F8
S1131B40794E8022346850012043802130600E0297
S1131B50D6E7754E8020346801012143802331602B
S1131B605E012BE0704C802120680B01034380222E
S1131B702360960122E06C48802301681A010A431D
S1131B8080260260F60119E0674880220368160186
S1131B901E4380240660260210E063488022036806
S1131BA01101194380240160E60207E05E488026A3
S1131BB00368310119438024016026030220311C8B
S1131BC0042202F095FA5A4803681E430660381E40
S1131BD0712800D062E72D68102050352F8801232A
S1131BE01F4268D0802B53D016D8082B47D009D871
S1131BF0022B3ED0042B3FD0012B00D0CBE080241D
S1131C00640052E0202B3DD0402B3ED0102B00D05E
S1131C10C1E08026740148E080252E01B34240D003
S1131C200FD880229400A34235D08021CD00AB424E
S1131C3034D080267200934200D0ACE0802464014A
S1131C4037E08026B20193422ED006D88024610169
S1131C508B4200D09FE0082427E08025EE01B342A8
S1131C6025D080221402A34200D094E080210C03EA
S1131C701FE08025AC0018E08021CC0015E0802115
S1131C800C0112E08024A4010FE08022D4010CE0B6
S1131C908022140209E08025AC010AE08021CC01F5
S1131CA007E08026340204E01024224E72E08025EE
S1131CB0EC02214E6EE0802B5AD014D8082B4ED063
S1131CC008D8022B45D0042B46D0012B63D18026A3
S1131CD074005AE0202B45D0402B46D0102B5AD10B
S1131CE08024640151E080210C01A34249D00ED824
S1131CF08025AE00B3423ED08022D1008B423DD03D
S1131D0080246500AB4246D18026740141E08024E2
S1131D10A501AB4238D011D88026720193423AD142
S1131D20082432E078F4FF1F38800440D4F00F40D8
S1131D3094F00F40C4F00F4084F00F408021CC0198
S1131D40A34224D080252E02B34224D1802214033E
S1131D501FE080218C0018E08022D40015E080224E
S1131D60140112E08026B4010FE08025EC010CE0A0
S1131D708022140209E080218C010AE08022D4012F
S1131D8007E080252C0204E01024064E02E08021A6
S1131D90CC02054E34605B0001389BB2002800D0B1
S1131DA01EE7F8BDC8F00F4088F00F4070B52E4B09
S1131DB0041C1A7850B2002830DB1D7802210D4231
S1131DC02ED11E78042216422CD1187885062BD4E5
S1131DD01E78012040251B78064203D02B4225D0D3
S1131DE0224934E02B4223D1214E3578054221D1BA
S1131DF03078084220D1317811421FD1327811074E
S1131E001ED43378301CDD061CD43678B1061BD4BE
S1131E10057869B2002919DA164918E0164916E05E
S1131E20164914E0164912E0164910E016490EE06E
S1131E3016490CE016490AE0164908E0164906E07E
S1131E40164904E0164902E0164900E01649002C40
S1131E5004D1081C04F052F8201C04E0201C04F0F7
S1131E6006F9041BE0B270BD00F007403FA100007A
S1131E7001F00740A49E000077A00000C49E00006B
S1131E80AA9C0000789D0000B0A00000B99C00004E
S1131E90FCB2000070A00000689F00004CA100008C
S1131EA0D19E00005AA10000A09E0000F0B50C1CB9
S1131EB091B0151C0B2801D900F001FD07F0B6FD07
S1131EC00C003B00A402C102FF0425039C04AF04E0
S1131ED0FF04FF04FF049F02081E05D0042907D154
S1131EE00120CA4908700020FEF760FE00F0E8FCFB
S1131EF002200529F5D003200629F2D00420072961
S1131F00EFD005200929ECD006200A29E9D00720C2
S1131F100E29E6D008200F29E3D009201029E0D0AB
S1131F200A201129DDD0122901D000F0C8FCB74BDA
S1131F3000201870D8E703921A2901D900F0BFFCD9
S1131F40081C07F073FD1B0027003401BC042101A9
S1131F50EA00BC04BC04BC04BC04CD00D7001E01D0
S1131F604800C4004A010D020D02BC04BC04BC04B8
S1131F70BC04BC04BC04BC04BC041F0001F0C0FFCE
S1131F8000F09DFCA24803F0B9FF0020FFF70EFF0C
S1131F9000F095FC9F4803F0B1FF9F4803F0AEFFAB
S1131FA09E4803F0ABFF02F0BBFB822103F0AEFFBF
S1131FB09B4803F0A3FF02F0A7FB822103F0A6FFD6
S1131FC0984803F09BFF02F091FB822103F09EFFEF
S1131FD0954800F06EFC002006A9471C02F0C2F9E7
S1131FE0924C061E45D0924803F088FF306803F0F7
S1131FF085FF904803F082FF0021079803F08FFFCC
S11320008D4803F07BFF8D4803F078FF00210A9888
S113201003F085FF201C03F071FF0021099803F0F1
S11320207EFF201C03F06AFF0021089803F077FF6D
S1132030834803F063FF0B98002103F070FF81488D
S113204003F05CFF0C9E002E03D10D9C301C002C71
S113205007D00D9B069D64206843F11807F0F0FC3F
S1132060C0B2002103F05BFF774803F047FF381C40
S1132070B2E7764803F042FF0C9D002D03D10D9B7F
S1132080281C002B06D00D9A64206843A91807F079
S1132090D7FCC0B2002103F042FF6D4803F02EFFCD
S11320A000210C9803F03BFF201C03F027FF0021C4
S11320B00D9803F034FF201C03F020FF0C990D98B9
S11320C04018002103F02BFF624800F0F2FB624845
S11320D003F014FF012261495042086000F0EFFB55
S11320E006A8FFF7DDFA002404705D4803F006FF3C
S11320F006A859E01778313F032F01D95948D8E38E
S1132100594803F0FBFE039A1078FFF7D7FB041E2F
S113211001D1564848E05648CBE31078011C3139C8
S1132120032901D95348C4E3FFF7C8FB002801D0B1
S11321305148BEE3041C01253120461CF7B2FFF7C9
S113214057FB002801D02C43E4B26800C5B2381E06
S11321503528F2D1039803F0B1FDC2B20398013AD5
S1132160012393400130DEB2039003F0A7FD012860
S113217001D1344300E0B443E0B20021FFF73CFC5A
S11321809DE3FFF76FFB9AE31778313F032FC9D81C
S11321903A4803F0B3FE039C2078FFF729FB041EA2
S11321A001D0374885E3374803F0A8FE47E1101C07
S11321B0049203F083FD051C04A8FEF78FFC00289D
S11321C001D0314875E3049A2F35E8B21178FFF74E
S11321D091FB002800D172E3F3E71078002802D1C4
S11321E01027009769E0101C03F068FD2749086078
S11321F003A8FEF773FC039E3378002BF0D04C2B1E
S113220001D06C2B44D104224DE0C04657F4FF1F8B
S113221050A6000064A60000D6A200007BA6000021
S113222001BA000088A60000D0A20000D5A60000D4
S11322309AA60000A1A60000ADA60000B7A6000063
S1132240D7A60000E2A60000F3A60000F7A600004F
S11322500EA7000046A9000012A7000000F5FF1F0A
S11322602AA700004FA7000061A7000074A7000080
S11322707DA7000085A7000094A70000A4A7000084
S1132280B1A70000B5A70000B9A7000038F3FF1FED
S1132290572B01D0772B01D1022204E0422B01D02D
S11322A0622B02D10122B94C2260701C0390757814
S11322B0002D95D003F01BFD0090B54803F01EFEE1
S11322C02020694608764876009E002E00DCF6E25F
S11322D0B04E8421306803F019FEAF4803F00EFEBF
S11322E06C461A341025A94A009B1768013B0093D9
S11322F0022F0DD0042F14D0012F00D0DFE230685C
S1132300013D0178013001913060081C11210FE07A
S11323103068023D0188023001913060081C1221AE
S113232006E03368043D04CB142101923360101C91
S113233003F0ECFD211C3A1C0198FEF7E5FB009F1D
S1132340041C002F09D10D260A2500232670657070
S1132350A37006A803F0D2FDB6E7002DC3D1F2E7BF
S11323601278002A00D1AAE2281C03F0A7FC051C5D
S1132370112C01D1894800E0894803F0BFFD03A86E
S1132380FEF7ACFB03980178002900D197E203F033
S113239095FC071C03A8FEF7A1FB0398814E037864
S11323A0002B01D1012017E04C2B01D06C2B01D163
S11323B004220AE0572B01D0772B01D1022204E03A
S11323C0422B01D0622B01D10122326001300390F3
S11323D0112CE7D103F08BFC3468002800DC6EE29A
S11323E0022C06D0042C07D0012C06D12F70013505
S11323F003E02F80023500E080C50138EDE7081CBA
S1132400111CFEF771FC5BE2002909D0032900D0FE
S113241055E26549101C0F6803F069FCF8834EE22D
S1132420624D2888042805D16148102603F066FD12
S11324302E8004E05F4B081C198000F0DFFB201C99
S11324403EE20592072900D939E2081C07F0E4FAB4
S11324500424474E1353583805A8FEF71BFB041CED
S113246005A8FEF717FB04A908700122201C02F03E
S113247067F951481DE205A8FEF70CFB061C05A8E8
S1132480FEF708FB4D4D04A92E4308700122B0B29B
S113249002F056F94A480CE205A804AFFEF7FAFA2E
S11324A0391C012202F06DF9002807DB454803F0CE
S11324B025FD3878092103F029FD00E24248F8E1BE
S11324C0394E42491822306803F03AFC404A3068D9
S11324D0116818303C2203F033FC3E48E9E1FFF771
S11324E0C7F80020FFF78AF83B48E2E1012002F038
S11324F060F93A48DDE1022002F05BF93848D8E19E
S11325000020FFF77BF83748D3E11D2900D9D6E135
S1132510081C07F08BFA1E00950032007800B10009
S1132520D401D401D401D401D401D401D401D401FF
S1132530D401D401D401D401CE00D401D401D401F6
S113254043014301D401D401D401D401D40157017E
S11325506B01154A00241768E100234B081B181867
S1132560291C03F06EFD002802D10337FC77A3E198
S113257001340C2CF0D11D489BE11778372F37D14B
S1132580094901200B689E8B064338E0D0F0FF1FF9
S1132590C1A7000038F3FF1FF8BB0000D2A700005A
S11325A0E0A70000D4F0FF1F78F4FF1F34F3FF1FEF
S11325B0EFA7000054F4FF1FFBA700000080FFFFFB
S11325C00DA8000025A800003AA8000085FBFF1F05
S11325D074F4FF1F5CA800007DA800009DA8000003
S11325E0B8A80000D5A80000B7A0000012AA0000F7
S11325F0382F06D1B34C012223689E8B96439E83C9
S11326005AE1B14855E1AF4B00261F68B200AF480C
S113261091194018291C03F014FD00280BD1B88B24
S11326200625A843002E04D0012E00D03FE1022449
S113263038E0042436E00136032EE7D1A44838E11B
S1132640A04F00243F68A34EA300F018291C03F0F8
S1132650F8FC00280BD1B88B1825A843012C04D012
S1132660022C00D023E110241CE008241AE00134D9
S1132670032CE8D198481CE1924B00261F68974927
S1132680F2008818291C03F0DCFC00280CD1B88B5C
S11326906025A843012E04D0022E00D007E1202497
S11326A000E04024204302E10136032EE7D18C48A8
S11326B0FFE08C4803F022FC8B4803F01FFC814CA4
S11326C023680333DA7F0B2A04D8D000874F861A95
S11326D0B81900E0864803F011FC864D281C03F06D
S11326E00DFC21682E1C8B8BDA0701D5824800E093
S11326F0824803F003FC824803F000FC22680123B3
S1132700908B810704D404273840454245416B002F
S113271099006E48CA18801803F0F0FB794803F05A
S1132720EDFB27680222BD8BE90601D42B07DA0FE3
S113273068489100401803F0E1FB734803F0DEFBA6
S11327402768BB8B0127590602D49D06EA0F570060
S11327506E4803F0D3FB6148F900401803F0CEFB48
S1132760301C03F0CBFB002F00D1A8E0684803F035
S1132770C5FB266800214C36307803F0D0FB654D4C
S1132780281C03F0BBFB644803F0B8FB2468002159
S11327904D34207803F0C3FB281C8AE0101C03F09E
S11327A0A6FAC7B2632F03D8002F02D1012700E095
S11327B06327444D2968152C01D14C3100E04D317B
S11327C00F7079E0554803F099FB554803F096FBE8
S11327D0012000F04FFF182103F0A1FB514803F042
S11327E08DFB002000F046FF18215DE001267042B9
S11327F000F040FF4C485CE0022909D004295ED176
S1132800304A291C10681422373003F099FA56E034
S1132810FEF7ACFFFEF78CF9FEF79CF94FE00A29AE
S11328204DD8081C07F0F8F806090C121E190F4BB6
S11328304B4B1500101C102111E0101C02210EE05E
S1132840101C04210BE0101C402108E0101C08217E
S113285005E08021101C890001E0101C2021FEF7F6
S1132860F7FD2CE0314803F049FB40213048FEF7E6
S11328707FF904212F48FEF77BF92F480821FEF742
S113288077F9002803D02D482021FEF771F92C4850
S11328901021FEF76DF9002811D02A4803F02EFB11
S11328A0084B08211868C08B03F039FB07E0B88394
S11328B002E003F023FB02E0042000F04FFA0020C2
S11328C011B0F0BD78F4FF1FEDA8000030A10000A6
S11328D02BAA00006C9D00003EAA0000F4A1000099
S11328E054AA000005A900001EA90000B7A000001A
S11328F026A90000ACB900002FA9000031A90000EE
S113290033A9000034AA00003BA900004AA9000032
S113291058A90000F3A6000064A900006FA90000F4
S113292084A9000095A90000A6A90000C1A900007F
S1132930D7A900001AAF000069AF000092AF0000F1
S1132940EBA90000F9A90000F0B585B003910021BE
S1132950071C029201910398002800D1F7E03B780C
S11329607C4C082B0CD17C4E3378002B05D07B4853
S1132970013B0130337003F0C1FA00222270E1E020
S11329801B2B04D05B2B05D122781B2A02D1237088
S11329900137D7E025785B2D4BD1181C413803282B
S11329A047D807F039F8101009026B490D78002D4B
S11329B000D1C7E0013DC4E067490D78272D00D957
S11329C0C0E00135BDE0664C28212068654E4143D6
S11329D0701803F057FB3B78051C412B08D1216884
S11329E0002901D1032100E0013921605E4806E09D
S11329F022680132032A00DD00225C48226003F0D1
S1132A007DFA002D04D05A4803F078FA013DF8E726
S1132A10564803F073FA206828256843301803F0F9
S1132A206DFA24686543701903F02CFB4A4E30702C
S1132A3088E00A2B00D185E0002B00D182E0484CCD
S1132A4028252168444A69431078464E0A1893554C
S1132A503B780D2B69D10A209055029800F062F959
S1132A602168444C4D4375193B4E0C20327826782E
S1132A70414946430132D3B28A197458E818567949
S1132A80029A013800210170002A05D13B480188CF
S1132A90002938D0490536D4002B31D0281C002E0B
S1132AA018D02168FDF7E2FF013E019000280FD005
S1132AB0334803F023FA207A617A019AFFF7F6F992
S1132AC0002801D1FEF7DCF8029B002B1BD112E099
S1132AD00C34E3E72B49FDF7C9FF021E10D0042094
S1132AE00921FFF7E3F9002802D1274803F006FA89
S1132AF0029D002D07D1214A108800F07FF802E0E2
S1132B00224803F0FBF900F01FF9154C124925681F
S1132B10002001350870032D03DC01262560019691
S1132B2006E001232060019302E00B4C0130207089
S1132B30094908480C78002202700137272C01D972
S1132B4027250D700398013881B2039103E701989A
S1132B5005B0F0BD3EF3FF1F56F4FF1FB59C000007
S1132B606CF3FF1FB4F3FF1F6DAA0000D1A2000095
S1132B70FBBB000057F4FF1F0CA200003CF3FF1F37
S1132B80ACB9000071AA0000BDA70000B9A70000FD
S1132B9008B50249182203F0D3F808BD01B30000B8
S1132BA070B5124D1248291C182201F0EAFD114E8D
S1132BB0002810DA0420291C182201F0E2FD002468
S1132BC0A0420ADA281CFFF7E3FF30680A493C22D6
S1132BD003F0B6F807E0802424021C202043316867
S1132BE03C2201F0CEFD201C70BDC04685FBFF1FBA
S1132BF00480000074F4FF1F50B3000008B5144BA8
S1132C00188020280ED004D800281CD008281DD1F4
S1132C1019E0802817D080214A00904208D040282B
S1132C2014D110E061200B49062201F05FFC0DE095
S1132C3096236120D900062201F058FC0648074A71
S1132C400178117002E0612001F08AFC08BDC046E1
S1132C503CF3FF1F7017000084FBFF1FE6F0FF1F0B
S1132C60F0B52A4C87B02A4E012822D1294D1822CA
S1132C70291C684603F064F8FFF792FF1822071C2A
S1132C80291C206803F05CF8326813899A071FD561
S1132C90281C04A90422103003F052F8281C03A9AC
S1132CA004220C3003F04CF8281C083002A904223A
S1132CB00CE0FFF775FF184D0422291F071C281C80
S1132CC003F03EF8291C20681439182203F038F860
S1132CD021681822114803F033F82068316818304D
S1132CE03C2203F02DF82068017E10290AD00C4CF8
S1132CF03C22211C183003F023F83068211C3C22AC
S1132D0003F01EF8381C07B0F0BDC04678F4FF1F6E
S1132D1074F4FF1F85FBFF1F99FBFF1F9DFBFF1F23
S1132D2050B3000000B5054B054A19781170FF2116
S1132D30002801D103480178197000BDE6F0FF1F97
S1132D40D8F0FF1F84FBFF1F024B03481A78027060
S1132D507047C046D8F0FF1FE6F0FF1F7FB51B4B3E
S1132D60011C1D68684600240472EA1CD67FC02238
S1132D70D300C672C38061222B1C40268680027356
S1132D804C331A782B1C42734D331A788273A88BF8
S1132D906A460090201C02F0BDFE0D4D2870A04232
S1132DA010D00521221C02F003FE0099314209D003
S1132DB00849221C287802F0FBFD28788121221C76
S1132DC002F0F6FD287804B070BDC04678F4FF1F09
S1132DD084FBFF1F0404000070B54F4C03302668C9
S1132DE090B0C57F002E40D13C2001F035FC4B4B08
S1132DF01860542001F030FC49490860301CFFF78A
S1132E002FFF80221602B04207D1962361201901B8
S1132E10032201F06BFB042000E001202060414804
S1132E2001F0EAFCFEF71CFE6D20042101F028FBF2
S1132E300320FFF793FF00286CD03B493B4E0A78F0
S1132E403B48327003F05AF87520042101F018FB56
S1132E504D20042101F014FB07E0062819D1324863
S1132E6034490078162203F029F8281C6946052203
S1132E7002F0B4FD00281ED06946CE780879002EF1
S1132E8002D0012E11D109E00328E6D101F091FC12
S1132E9001E08328E9D101F033F8E6E7DD28E4D145
S1132EA02268082AE1D12660DFE7021C6946281C53
S1132EB002F094FDD9E7246837252C422AD01A4C15
S1132EC0207802F09BFD002824D020786946402217
S1132ED002F084FD061E1DD06846311CFEF74EFB31
S1132EE01548311C02886846002A0FD1FFF72CFDD3
S1132EF00028EAD080235800FEF746FC0228E4D1DB
S1132F0020780E49172202F0D9FFDEE70022FFF7EE
S1132F101BFDDAE710B070BD7CF4FF1F74F4FF1FD3
S1132F2078F4FF1F20B3000084FBFF1FE6F0FF1FAF
S1132F30A3B300008CB300003CF3FF1F58B800009B
S1132F4070477047704770477047704770477047C5
S1132F507047704710B50D4B0D4A187811785F23F0
S1132F600840041C9C4310D0820607D509480A4A2D
S1132F70017890780840022102F034FC63B2002BFF
S1132F80E9DA022002F0ECFCE5E710BD04C00640DB
S1132F9003C0064007C00640D8F4FF1F10B50D4B10
S1132FA00D4A187811785F230840041C9C4310D004
S1132FB0820607D509480A4A017850780840012159
S1132FC002F010FC63B2002BE9DA012002F0C8FC25
S1132FD0E5E710BD04B0064003B0064007B0064064
S1132FE0D8F4FF1F10B50D4B0D4A187811785F23E4
S1132FF00840041C9C4310D0820607D509480A4A9D
S1133000017810780840002102F0ECFB63B2002B39
S1133010E9DA002002F0A4FCE5E710BD04A00640B4
S113302003A0064007A00640D8F4FF1F054B10B5C7
S11330301C682188002900D10349018001F082F92C
S1133040208010BDB8FBFF1F7B120000074B0C2033
S11330501A6800B5024204D005495523AA220B6020
S11330600A608020034B0106196000BD0081044002
S1133070048104400CF10F4072B6024B1A6801320D
S11330801A60704794F4FF1F044A00B51368013BAB
S11330901360002B00D162B600BDC04694F4FF1F3C
S11330A03B4BF7B5141C1A68051C1F1C002A12D1CF
S11330B0384A01208243161C3C36131C00963648BD
S11330C0861A188801969853009E0233B342F6D1AB
S11330D0314A01323A60314E337858B20028FADA74
S11330E0327830231A4200D033702D480570092DF0
S11330F018D002D8062D2FD114E0412D29D0432D0C
S11331002AD10968274A284B1170E078274A187099
S11331106188274B11702068264A010A19702068BB
S1133120107019E01F480A0C0270234B23480A0A46
S11331301A700170062D0FD1E1781B4A1B4B1170D8
S11331406088187021681A480A0A0270194B2168AD
S113315001E00968134B1970FFF78EFF0F483F68B1
S1133160B847FFF791FF412D0ED10F4D0F4A2B7831
S11331701078190607040F430E4D0D492B780A7871
S11331801F43100207432760307831242040FEBDDE
S113319084F4FF1FDAF0FF1F98F4FF1F00000240C1
S11331A007000240060002400B0002400A000240F1
S11331B009000240080002400500024004000240E9
S11331C008B58022044B90041860FFF755FF01F006
S11331D0EFF9FFF759FF08BD04ED00E0F7B50F1C48
S11331E00090161C1D1CFFF747FF00980C23584342
S11331F02C4901900A682C4C13189868A360430664
S113320002D4291C103101E0291C183161600431F9
S1133210E160381C7168009A231C01F0F3FD071E5D
S1133220032F07D0042816D0012829D1FFF72CFF3B
S1133230381C36E0A36861685A6880273A430A60FC
S113324058689C6840256840654058609D603368B4
S11332501F43376022E0009A002A04D184202861A9
S1133260A861101C09E0009802F09EF80F4D43017C
S113327029688422CF183A61BA61082102F088F8DB
S1133280084D019B29680A4ACF18B868256802408E
S11332902A4322608024144334603A60FFF7F4FE2A
S11332A00020FEBD90F4FF1FDCF4FF1F80F4FF1F1D
S11332B00800FF03F7B5A24EA24D33782C781C40CA
S11332C000D13BE10821201C884300D187E001277D
S11332D0FFF7D2FE3C424BD09B4A33233370117824
S11332E0022739431170287830239843974928706E
S11332F00968402388689843002388600B6011782C
S11333009348B9431170934A9349012713700F707E
S1133310924A0370924F9348137013703B7003707A
S1133320914F92483B700370914F92483B700370E9
S1133330914F92483B700370914F13709148924A99
S113334013703B7003700B7804201F1C0740FAD1E4
S11333508E498F4A0B688F499A6019603A1C391C50
S11333608D4B01F04FFD8C487B4B87740D271F70EC
S1133370A10712D5894B1A78570703D588484168A5
S1133380013141601F78B80703D5854A10680130C0
S113339010600621197002233370E1060BD5302723
S11333A03770287820221043002128700A1C052039
S11333B00B1C01F027FD20210C420AD0302333706E
S11333C02F7806208F4300212F700A1C0B1C01F05C
S11333D019FDFFF759FE0825221CAA433270082064
S11333E0044200D167E76F4A684C137821681C09CE
S11333F06701CB191778684D074220D00C2262432D
S1133400524F396888188268A860570604D4191C7A
S113341010316960143303E01F1C18376F601C33CC
S1133420EB60FFF729FE221C2B1C0021032001F076
S1133430E9FCFFF729FEAC7C464D2C707BE010784C
S1133440042210401A1C002801D0083240202860B1
S113345010688701BF0D2F823C273840042802D012
S1133460342861D129E00C276743384D0197296836
S1133470C91988688027000701D509680F403648B4
S1133480A10009180878C00602D5201C012101E01A
S1133490201C0221FFF7A2FE2B68002F06D0019901
S11334A05D18286880239843021C04E0019C802254
S11334B01D192F683A432A603DE02D680020AC4670
S11334C0186198610C276046204D6743400609D473
S11334D02868C719BF6834483840C0270860384393
S11334E0886008E02868C719BF682F483840C0279B
S11334F08860384308600C27674329684820C91945
S1133500486011492020097881430F480170201C2C
S11335100021FFF763FE01280DD02B688022DC19FF
S113352025682A43226006E0842119619961201CE0
S1133530082101F02DFF08233370BCE6F7BDC04617
S113354080200740842007409420074090F4FF1F08
S1133550C420074098200740C0200740C8200740E7
S1133560D0200740D4200740D8200740DC20074063
S1133570E0200740E4200740E8200740EC20074013
S1133580F8200740FC200740F420074080F4FF1F88
S113359088000800C8000800DCF4FF1F88200740EA
S11335A088F4FF1F902007400800FF03104A114BC6
S11335B011481A601149124BC863F02219681005AA
S11335C0084318600F4B104807221A6003688021D3
S11335D00A041A430D4902600D4B002008600122C1
S11335E00C4918605042012208601A607047C046B6
S11335F0FF9E240014E000E0C131000000F0FF1F32
S113360020ED00E010E000E03C8004400070034046
S11336101871034010710340134B021C10B5802431
S11336201968A243530140B2CB18002813DA0F499A
S113363094000C20611842430D4C20688218546891
S113364040208443546000221A619A610B7802245A
S1133650A3430B7006E019689A680424A143A243AB
S113366019609A6010BDC04680F4FF1FC020074057
S113367090F4FF1F08B5002809D001280AD00130B2
S11336800BD100210822064802F051FB05E0044852
S1133690006803E0024B586800E0002008BDC04603
S11336A088F4FF1F38B5184A0C1C1849031C800005
S11336B01568421811780120490723D50C20144AB3
S11336C0584311685B010818A060ED18FFF7D4FC9B
S11336D0A26891684A0604D42B1C10336360143525
S11336E003E0281C183060601C35E56064688022A3
S11336F02568154003D0FFF7C7FC022002E0FFF75E
S1133700C3FC281C38BDC04680F4FF1FC0200740FE
S113371090F4FF1FF0B5384D161C8A0057193A78FB
S11337200C25AA434D439C46344B85B01C684B0181
S1133730334903953A70E418039A0B6801979B1870
S11337400027A7612761A76027602E4A9F601F603A
S1133750FF2806D1157830239D431570019A177000
S113376047E011781025294311708022011C9143F0
S11337700291012902D15F60242503E008275F60DC
S11337800525482740B200282EDB6368002B0CD1A6
S11337906246B44500D2321C96B2301C00F05CFF85
S11337A06060301C00F058FFE060174B31040B40A0
S11337B080221F43161C40213E438F433A4322601C
S11337C0A6600F4C039A236808209E18B760029FD6
S11337D02843002F01D1051C03E004208543182150
S11337E00D43019C257004E0029E002EF9D01021A7
S11337F0F6E705B0F0BDC046C020074080F4FF1FC7
S113380090F4FF1F842007400000FF03F7B50C2647
S11338104643184F184B3A681C6893594101402598
S113382064182B4202D00021009101E00834009575
S113383022688025131C2B40019301990123002940
S113384016D19201920D616801F05EFA02230128FB
S11338500ED03868094F8619B36800991F400F438A
S11338602A1C3A4322603468019B25402F43376069
S1133870181CFEBD90F4FF1F80F4FF1F0800FF0317
S1133880F7B54B4B4D7C0C1C4A4A196880200A4002
S1133890060632431A60277C0135EDB2012F05D1AB
S11338A0454BA0211A68CF02174308E0434B8022FE
S11338B01968900108431860E026414BF70041481D
S11338C01F6003688026F7021F43E9B207601029CE
S11338D000D91025EDB20C20684300F0BDFE3A4E2D
S11338E080223060394807783A430270374B1978A0
S11338F048B20028FADB364F022280213A70914008
S1133900680100F0CDFE334B334D010A2860197075
S11339103249020C0A70324B324A0021000E1870F0
S113392011703970304F3970387804231840019081
S1133930FAD108202F6800F08FFE786008202F68E5
S113394000F08AFE2D683668F8602849284A29481C
S1133950254B0D272A60A960B06027491F70274EA8
S1133960274FED25FF22BF200D70264B3270264DC8
S113397038708021254E264F4A0460201D60326035
S11339806B4638701979234D234E244F104B297000
S11339908B2206200125327038701D7064892C42F8
S11339A005D00A491E48402210260A700670F7BD49
S11339B000700440FFFFFFBF0480044038800440CF
S11339C068D004403480044090F4FF1F0C21074069
S11339D0942007409C20074080F4FF1FB02007403C
S11339E0B420074098200740C02007408800080002
S11339F0C800080008000800102007408020074085
S1133A0088200740A0F0FF1FB532000000E100E06D
S1133A1018E400E000210740842007408C20074080
S1133A2008210740274B820030B5D358012817D00E
S1133A30002805D0022844D18024234A640112E0DE
S1133A40214A8025EC0015682C4314601F4A204C41
S1133A5015682C431460CA7A0B2A0DD99D220EE0F6
S1133A608024194A240115682C431460CA7A0B2A4D
S1133A7025D85500174C01E0174C55002A5BD50496
S1133A80EC0E1C705A700A68144C0621D50709D52F
S1133A907F252554114010D0510701D503200AE099
S1133AA0022008E0FF252554114006D0540701D513
S1133AB0132000E01220987003E0997001E04F2277
S1133AC0DDE730BD3CB9000034800440048004408C
S1133AD00000010448B90000D8B80000D8F4FF1F62
S1133AE0234B820000B5D358012829D0002815D0D3
S1133AF0022837D11F4A802110684901014311600F
S1133B00C0221D49900008601C4A1D48802190670E
S1133B101C4AC8011060A0211B4822E015498022DC
S1133B200868920010430860184919480A60134A4B
S1133B3080211067134A48011060C021154810E025
S1133B400C4980220868920110430860C021880053
S1133B50114908601148094948670A48B0210260C0
S1133B600F480170DA7808210A43DA7000BDC046B4
S1133B703CB90000388004400CC0044000F0FF1F32
S1133B80552F000000E100E00EE400E0089004403E
S1133B90E52F00000CE400E000D004409D2F00005D
S1133BA00DE400E0034B8000C0587722C1780A403E
S1133BB0C27070473CB90000234B820000B5D35853
S1133BC0012829D0002815D0022837D11F4A802186
S1133BD01068490101431160C0221D49900008602A
S1133BE01C4A1D48802190671C4AC8011060A0210E
S1133BF01B4822E01549802208689200104308609F
S1133C00184919480A60134A80211067134A480169
S1133C101060C021154810E00C4980220868920108
S1133C2010430860C02188001149086011480949FF
S1133C3048670A48B02102600F480170DA782421ED
S1133C400A43DA7000BDC0463CB900003880044025
S1133C5008C0044000F0FF1F552F000000E100E001
S1133C600EE400E004900440E52F00000CE400E0C2
S1133C7004D004409D2F00000DE400E0034B8000BD
S1133C80C0582421C2788A43C27070473CB90000EE
S1133C90034B8000C0587F22C1780A40C27070472D
S1133CA03CB9000000B5084B8000C35801201A79C4
S1133CB052B2002A06DA8020D971D97842420A43E6
S1133CC0DA70002000BDC0463CB9000038B5840A53
S1133CD00D18A4020920211C0022FFF7E1F9002895
S1133CE006D180232A1BD9008A4202D96418F1E73D
S1133CF0012038BD08B58021C900FFF7E7FF08BDE2
S1133D00F7B503230191161C204C002909D1206822
S1133D10184201D1002038E098430421206000912A
S1133D2004E0021C9A43184022600090009F04257E
S1133D30ED1BB54200D9351C154A009B0199D718D3
S1133D40381C2A1C01F0FCFF0198114B41197A1907
S1133D5004330191761B9A4210D3062021680C4A41
S1133D60FFF79EF9071E0FD12068FF210430206061
S1133D700422074801F0DBFF009702E027687D1961
S1133D802560002ED2D1C5E70120FEBDF0F4FF1F4F
S1133D90D4F4FF1F37B5C421051C49026846082224
S1133DA06B425D4101F0CCFF0D4C009B6D422543FD
S1133DB0A34202D10198A8420FD0C62251026846FC
S1133DC0082201F0BDFF00990020A14206D1019C08
S1133DD0631B5D426B41580000E001203EBDC046BC
S1133DE055555555F8B5151C1E1C022801D0C42480
S1133DF000E0C6246002083089004418281C7219A7
S1133E0097B283B29F4207D0471C211C012201F0C4
S1133E1097FF0434381CF2E70020F8BDF0B585B0F4
S1133E200193002543B20E1C0092AB4202DA7F21BB
S1133E3008400125410608D5C4204002FFF75AFF77
S1133E40C6225002FFF756FF02E0C624022800D023
S1133E50C424019F6402002F05D0231CB60008333C
S1133E609F19009E11E0002D09D0C421480284420C
S1133E7001D1C6235802FFF73DFF002518E0201C9E
S1133E80FFF738FF002E13D033E001990098B3B246
S1133E900A1891B299420BD03078174A03A91043FB
S1133EA003900422381C0136FFF72AFF0437ECE79D
S1133EB003A8211C042201F043FF104E039FB742C4
S1133EC005D0201C03A904220396FFF719FF002D37
S1133ED00FD1043403A8211C042201F031FF039DF7
S1133EE0B54206D0054803A903900422201CFFF71D
S1133EF007FF002005B0F0BD00FFFFFF55555555E5
S1133F00024A034B00B51A60FEE7C0460400FA05F6
S1133F100CED00E010B5124A12490023891A8B42B5
S1133F2004D01148C45CD4540133F8E70F49104A53
S1133F30914204D10F4B104A991A002308E00F480C
S1133F400023801A8342F5D0CC5CD4540133F9E7C2
S1133F508B4204D0D018002404700133F8E710BD5C
S1133F60C0F0FF1FF3F0FF1F80BC0000100400002E
S1133F7010040000C0FBFF1FF4F0FF1FA09B000013
S1133F8008B5394B802219689000084318603749F6
S1133F90374B384819600168374A384B0A40026089
S1133FA0186880214A010240354B00D00C221A6067
S1133FB03449354B9822942008701A701A1C334BDC
S1133FC018788007FBD51978C806FCD418780C211A
S1133FD001400829FAD12E49032008702D495820A0
S1133FE0087018788006FCD519784806FCD52A484C
S1133FF02A4908602820107019780C220A400C2ADB
S1134000FAD1274B27482849284A0360D9601A6106
S113401027482849284A586199611A63274828493A
S1134020284A98609963DA62274B2849284A181C61
S113403002C39042F9D1FFF76DFF0422FF21254806
S113404001F075FEFEF77CFF2348244B24491860D9
S1134050244800F0DBFA24482449092200F0AAF895
S113406000F0B0F9FCE7C0463880044003010010BA
S11340708090044014F00F40FFEFFFFF10F00F405A
S113408000810440014006400040064006400640CE
S113409004400640054006400000011044800440EE
S11340A000F0FF1F08ED00E0432F0000452F000043
S11340B0472F0000492F00004B2F00004D2F000018
S11340C04F2F0000512F000040F0FF1F532F00001E
S11340D0BCF0FF1FD4F4FF1FFC2F0020B8FBFF1F10
S11340E0C0FBFF1F70B8000078B8000032B90000B0
S11340F010B5084BC01800030123002909D0194248
S113410004D08024640014430460994304305B00A9
S1134110F3E710BD490004001E4A30B51368101CB3
S1134120002B35D01C4900250C681C49E2430124AE
S11341300D6065421A4C256001250D6059698A425B
S113414000D25A611C69A24203D9164D1A6129682A
S11341509961DC689D68A2180135DA609D600023CE
S1134160036011480468011C621C11D10F4A1068D5
S11341700568002D09D00124002562424261856052
S11341800561C56085612830F2E7094B0D601D604B
S113419030BDC04608F5FF1F147103401871034079
S11341A010710340BCFBFF1F00F5FF1FF4F4FF1F59
S11341B0FCF4FF1FF0B587B003905C4805925C4F98
S11341C05C4A0023057813603B600C1C2678002EA3
S11341D04FD076B2AE4245D1221CA01A002601343B
S11341E0A657C5B2002EF8D128206843043000F049
S11341F033FA3860EF43E419A446341C61464B7823
S11342000193002B2BD0039B1968002924D00F782D
S11342106A4604971779049A7FB2BA421AD15F6842
S11342200160476019898183002901D00136F6B203
S11342305989C1839A8902849F7B031DDF770127F3
S11342407B424361002901D1002A01D00134E4B248
S1134250283001E01033D7E701218C44CEE7019ADE
S1134260026008E0013400216356002BFAD10134C6
S1134270ACE7341C351C2E4F386800284AD0002C7B
S11342802CD00C216143043188B200F0E5F9294AAD
S11342903B6810609446196800291AD0DA8B002A0A
S11342A007D025498A4201D10022DA83D98B4160A3
S11342B003E0198C002901D04160012241680029E2
S11342C001D001214172002A01D003600C3028334F
S11342D0E1E70C235C43041B60460460059AB118B3
S11342E0C8B201F057FB002E14D03C682668002E9B
S11342F010D0A08B00280BD001210320221C01F038
S113430009FC211C22310870002801D1FF220A7007
S11343102834EBE70948FEF789FE094B00271F60A4
S1134320FFF744F9281C07B0F0BDC046D9F0FF1FC1
S1134330F4F4FF1F04F5FF1FFFFF0000F8F4FF1F54
S1134340BCFBFF1F054A06481188CB07DB17034057
S113435049084B4098B210807047C046F8F4FF1FDC
S113436000B4FFFFF8B5154B071C0C1C081C2022D9
S1134370002100261D6801F0DAFC301C2A68002A9E
S113438016D0EB68F618002F0FD1A96861600029D8
S113439008D02869A0606A69181C2261236005F0AE
S11343A04FFBE060A969281C61612835013FE5E7FE
S11343B00349A6610D68E561F8BDC046F4F4FF1F2A
S11343C0FCF4FF1F274B73B51C682334261C233EC3
S11343D03268002A45D020780D2108423DD0224D74
S11343E0224A2B680020106001212148DD434B4202
S11343F00121036011601F4A13689D4200D91560B2
S11344001D481E4A016816606D180560FEF734FEEB
S1134410E31E1888002802D12178CA0716D46378CD
S1134420002B0ED000256A46157055703068694619
S11344300278281C8A700522CD700B7101F03EFDB4
S1134440657021780A230B4000D12370251C1F3D81
S1134450FEF71AFE2A68301C9047FFF75DFE2834E9
S1134460B4E773BDF4F4FF1F1471034018710340E3
S11344701071034000F5FF1FFCF4FF1F08F5FF1F38
S113448038B5174B1C682268002A28D01578854255
S113449023D1002919D113480568002D15D02B68A4
S11344A0002B12D09C420ED1FEF7E6FD218C002990
S11344B003D00D480368CA186A6004340025E57700
S11344C0FEF7E2FD0BE00C35E9E704344A0702D5B8
S11344D0E27F120703D4E17701E02834D3E738BD43
S11344E0F4F4FF1F04F5FF1FBCFBFF1FF8B5194BC5
S11344F00E1C1C68171C002C2BD017490D682A6849
S1134500002A26D01378834221D12068002820D0A5
S113451085421AD1FEF7B0FD2B1DDA7F02218A43B2
S1134520DA772772002F04D12E84002E04D166720C
S113453008E0002E00D101260848012305686372B3
S113454077196760FEF7A0FD03E00C34DDE728353A
S1134550D5E7F8BD04F5FF1FF4F4FF1FBCFBFF1FF4
S113456038B5114B1C68002C1DD010490D682A6801
S1134570002A18D01378834213D12068002812D05F
S113458085420CD1FEF778FD002121726172043559
S1134590EB7F02221343EB77FEF776FD03E00C3446
S11345A0EBE72835E3E738BD04F5FF1FF4F4FF1FFC
S11345B0144A154B11681B68013130B51160141C85
S11345C0002B1ED01A68002A1BD0587A002816D057
S11345D0256859688D4212D1111DC87F850706D4FC
S11345E0050701D40425CD77187A511DC877128C9C
S11345F0002A03D05D68A818586000E05A720C3392
S1134600E0E730BDBCFBFF1F04F5FF1F13B50E4BE5
S113461000221A800D4C0E4B0E4A2160196014784A
S11346201A1C0378A34203D0002B0CD00430F8E703
S11346304088091811606C460734A14203D85522FA
S11346400A700131F7E713BD10F5FF1F0CF5FF1FCA
S113465014F5FF1FD9F0FF1FF8B50E4F0E4E3B683F
S11346603488051C1C190320044201D084430434FB
S11346700A4A611913688B4209D92A1C201C00219B
S113468001F055FB3F68E01B2D18358000E0002445
S1134690201CF8BD0CF5FF1F10F5FF1F14F5FF1FBC
S11346A0F8B50F4F0F4E3B683488051C1C19481E83
S11346B0044202D04A42144064180B4B6119186832
S11346C0884209D92A1C201C002101F030FB3F68D4
S11346D0E21BAD18358000E00024201CF8BDC04664
S11346E00CF5FF1F10F5FF1F14F5FF1F054B00B558
S11346F01A68131C981A0133197880B25529F9D015
S113470000BDC04614F5FF1F034B044918680A682E
S1134710831A98B27047C04614F5FF1F0CF5FF1FAB
S1134720044B05491868054B0A681988801A421A0F
S113473090B2704714F5FF1F0CF5FF1F10F5FF1F13
S113474070B5041C01200E1C151CFFF723FB002868
S113475007D1FFF71FFB002800D141200323584055
S1134760C0B221B2002905DA802253421843C0B2F4
S1134770032148406404321C2B1C610CFFF74EFBE0
S113478070BD03B270B5041C0E1C151C0120002B57
S113479002DA6404640C0020FFF7FCFA002805D058
S11347A0211C321C2B1CFFF71DFB01E001204042A1
S11347B070BD08B5022804D003280ED0012817D1F3
S11347C00CE00020FFF7E6FA002811D080235942BC
S11347D008430021C0B20A1C06E00020FFF7DAFA01
S11347E0002805D001210022131CFFF717FB01E06C
S11347F00120404208BD0000014B18607047C046CC
S113480018F5FF1F08B5FEF721FC08BD10B50028F8
S113481009D08069431DDA7F141C0C34640000192C
S113482001328180DA7710BD10B5831CCC0706D520
S11348300478148040780002044314800232981CE7
S11348408C0706D51C7814805B781B021C431480EB
S113485002324B0705D504781480417808020443DA
S1134860148010BDF0B58BB0051C68462630059148
S113487006921C1CFCF7DCF8021C01200021844673
S1134880137803936B46DF8C039EB81B87B204979F
S11348901020C75ADF845378042B0FD0052B20D067
S11348A0022B41D15179491B4B425941002901D175
S11348B0002D39D100260121B44635E0002933D03A
S11348C0059EFF2E02D09378B3422DD10698FF287F
S11348D003D0D7780321874226D1002C2FD0022180
S11348E022E0002920D0002C1ED08F1E784278416F
S11348F00190231C1868002812D086789778774096
S11349007F060BD1019E002E0ED1477900793E021D
S11349109F883043874207D2988005E00833E9E74F
S1134920019E002E00D01A60039E049B9219002B56
S1134930A6D161464D424D416842204000E0101C22
S11349400BB0F0BD70B5041C80780B1C7F22011CD9
S1134950114028254D430C4E90433668E278751972
S113496066791043320226793243FEF7D3FEE078AB
S1134970AB1C002801D1112403E00335EC7F012195
S11349800C43DC7770BDC04620F5FF1F37B5836943
S1134990051C0133D87F002813D02A8A8A4210D8F4
S11349A06946002488700123DD2008710C704C7066
S11349B0CB70201C6946052201F080FAAD690135EF
S11349C0EC7737BDF7B5282401935C43364B009050
S11349D01868089E0419E58A0020854262D1228362
S11349E0131C8A4200D90B1CA28A9FB2E38297420D
S11349F001D9628200E06382F0680099658A0160EF
S1134A00B36880205A6829041043284A114001439E
S1134A10706840220160986859685140424059606A
S1134A209A60E068291CFFF7F1FE009B6360E28A4C
S1134A30618A8A4207D0E068002806D0836905337A
S1134A40DA7F012A01D9E08A2CE00198311CFEF7B3
S1134A5029FE0028F7D100997F1B4D190095A08AE3
S1134A60BFB23B1C874200D9031CF26800999DB277
S1134A701160B36880205A68290410430B4A11401E
S1134A80014370684022016098685968514042406F
S1134A9059609A60E068291CFFF7B8FE638AEA1837
S1134AA06282C4E7FEBDC04620F5FF1F0000FF037D
S1134AB0F0B58BB01C1C10AB03900F1C161C1D789A
S1134AC0FEF7DAFAA01E042800D992E04C492A0124
S1134AD00C68A31804F0A0FF031A67178200F804F7
S1134AE001D59D6800E05D68710608D5AE69B11C0A
S1134AF0C87FC00703D57F231F400136F777AF690E
S1134B000237FC7F76E05868048A73E09D68002DC4
S1134B100CD1039805A9FEF7C5FD2C1C002869D10A
S1134B2005AC0094381C311C321C37E0AC690234EB
S1134B30E17F0024CA075DD5A74206D1E88A2B8A03
S1134B40C21AB24256DB94B254E0FEF79DFA391C05
S1134B50321C281C01F0FDF8061C041CFEF78CFA1C
S1134B60AF690237FB7F40273B4243D1039805A935
S1134B70FEF798FD00283DD1EA686868141AAA690E
S1134B80A3B20232D17F0F43D777371C9E4200D99C
S1134B901F1C6868BAB205AD0095111C039BFFF792
S1134BA011FF041C26E05D68391C321C281C01F02E
S1134BB0D0F9AF6904260237F97F041C31421BD0B7
S1134BC0FEF75AFAAB690233DA7FB243DA77A8699F
S1134BD0807EFEF71BFE0028F9D00BE0002E01D0EA
S1134BE09D6800E05D682A680024AA606A602C82DF
S1134BF000E00024FEF748FA201C0BB0F0BDC046CC
S1134C0040F5FF1F38B5011C7F23194028244C436D
S1134C100E480268FF2014190022131CE568FEF7F1
S1134C2079FD0023A11C601DCB77E382C3779D42ED
S1134C3003D02A682B82AA606A60A468002C04D07E
S1134C40216800252582A160616038BD20F5FF1F21
S1134C50F7B5051C294F1C230430A97B284A3C685E
S1134C6000F00AFF0190AE7B2823002E0AD05E4399
S1134C70A419AE89A6826B89DA0613D5E01C20221A
S1134C80C2770FE0687C01305843FFF7E5FC041C51
S1134C9038600820A082AA7C611CCA77301C291CB9
S1134CA0FEF7EEFD0199174B013918680E018219C0
S1134CB09168E160002902D08C612E892682AB7B49
S1134CC0A376A87B00280CD0EE7B002E09D02824E4
S1134CD074433F683C19A676A97B231DD977A8891C
S1134CE0A0825268A260002A03D09461AE7C671C43
S1134CF0FE772D6801982560FEBDC04620F5FF1F94
S1134D00B14A000040F5FF1FF0B50E1C2821151C08
S1134D1048431B4A85B0146824182768002F03D120
S1134D20A068002807D129E0301C291C1A1CB847A8
S1134D30072823D1F4E7631CD87F002803D040B2AE
S1134D400421FFF79DFBA3680234E27FA44601928D
S1134D50019C04210C400120002C0FD1DA8A1F8A07
S1134D60D21BAA4206DB181C311C2A1C00F0F1FFDE
S1134D70201C03E0019E65460E43EE7705B0F0BDAE
S1134D8020F5FF1F70B5A0B00E1C80220021051C69
S1134D90684600F0CCFF301CFF2100226B46FFF771
S1134DA061FD002828D000246B461859002824D01F
S1134DB0002D0BD1002E03D18078FFF723FF19E0DB
S1134DC000AB1A199188FFF7BDFD13E081787F20AD
S1134DD0084028230A4A5843126810180230022255
S1134DE0C17F012D01D1A94302E091430A1C012195
S1134DF00A43C2770834D7E7012020B070BDC0460B
S1134E0020F5FF1FF0B5ABB00D1C05921F1C00244C
S1134E10062800D9AEE204F009FE2F0186028002C2
S1134E2007008D029D02A402059B28255D43BF490E
S1134E3008684619F58AF468002D1BD1002C00D1AE
S1134E4098E2268A002E0ED06368E268934202D369
S1134E50E08A191A61606068131A9DB2B54200D9DC
S1134E60331C9AB295E0A46940250234E77FAF432E
S1134E70E7777EE2728AAA4200D2B6E0002C00D123
S1134E8092E0228A9446002A00D18DE0A3699A8B8D
S1134E90581D06920390C17F0122049104980233A5
S1134EA0824207DA988B694607901C20415A0132E6
S1134EB05983F3E70699039B01386246D877501A61
S1134EC083B2069369461822505AA2692082131CA1
S1134ED007920533D87F41004B42023B04934000C4
S1134EE0002310181A1C0499023B8B4205D0C118E8
S1134EF0898B8C46624492B2F5E7069B934234D187
S1134F00002B4BD1059A002A04D0B01CC17F30235A
S1134F10194215D0B18A281C04F0D6FD8AB2002AA1
S1134F200ED1BB68882158687F68014339605F6887
S1134F309968402257404A405F609A600123069373
S1134F406068E26845196560954202D3E78AE91B07
S1134F5061600023F382069E9E421FD1079840227F
S1134F600230C57F9543C57718E06068E36845194A
S1134F7065609D4202D3E18A681A60606068069D9C
S1134F801B1AAD1A99B2AAB28D4200DB0A1C002387
S1134F90F3820097111C059BFFF714FDA669201CE2
S1134FA0318AFFF7F3FCE4E1B18A281C04F08CFD9C
S1134FB08CB2002C16D1338BAB4206D1059D002D4B
S1134FC010D0B01CC17FC8060CD4BC6888226368AA
S1134FD07F681A433A606068A168402568404D4084
S1134FE06060A5600024F482C4E1AD1AB38AA9B25A
S1134FF0994200D91D1CADB2002C1FD0A3695A1DC3
S1135000988B0792D17F8446069101220698023339
S1135010824207DA998B142005916946415A01327C
S11350205983F3E7079B0138D877218A6246881AA7
S1135030A3692082198A201CFFF7A8FC728A706871
S1135040F96883180B60BB687A685F688020384908
S113505038432F0439400143116058689F68402247
S113506050407A405860291C201C9A60FFF7CEFB00
S1135070748A2D1975827CE12C4A0C78166880217B
S113508000208C43F0820594012C00D188E0022C8E
S113509000D1FDE0002C00D08BE06878092800D90D
S11350A087E004F0B9FC78868686863F05867447D7
S11350B0EC78A978EB792002AA7908431C021443FE
S11350C0031CFF228021934389008B4213D0C0210B
S11350D089008B4215D08020420093421AD16D463C
S11350E02235281CFBF79EFC2988221C00970023EC
S11350F0FFF768FC3DE16D462235281CFBF798FC60
S1135100F2E76D4622351040291CFBF797FC002876
S1135110EAD18AE036680424002E00D12AE1681C12
S1135120398A4DE0AE789E748CE0C04620F5FF1FAE
S11351300000FF03A978914F00203970FFF722FE89
S1135140061E02D000263E706FE08D4B1C680134B1
S1135150E27F03240592002A00D10BE16846A91CD2
S113516001222E3000F0ECFD6D461420415D0AAFA3
S11351700222B97075233A71FE25301C391C0722AE
S11351803E707E70FB707D7100F098FEF2E000933B
S11351907A48012102E07B48009302210A1CA6E719
S11351A06978A81C0691002967D00A294CD00B29DC
S11351B00AD036680424002E00D1DBE0398A281C8A
S11351C00022B047041CD5E06C4F04243B78002B2C
S11351D000D1CFE009AC0321221CFFF725FBA57801
S11351E0002180220AA800F0A2FD3878291CFF22A1
S11351F00AABFFF737FB002608360AA88219083ADB
S11352001568002D03D0A878FFF7FCFCF4E7A67816
S11352102478291C802200F08AFD3878311C221C55
S11352200AABFFF71FFB002801D10424A2E00AA85F
S113523008354719083F3868002803D00021FFF7D4
S113524081FBF4E7032495E04C4D042429780029DC
S113525000D18FE06E4622360221321CFFF7E4FAB9
S113526028783178059A0023FFF7FCFA002800D14A
S113527080E003300097059990E7404B04241A78A6
S1135280002A77D0022100973F480A1C069B2FE78B
S11352906C780694012C38D8A81C6D4622350599E3
S11352A02A1CFFF7C1FA354B1978002903D1288845
S11352B0042400285ED12C881F22224028256A431A
S11352C00699B01802300823012914D1C77F1F4260
S11352D04FD09F433368C777002B4AD0E0B26C4667
S11352E021342070FEF798F9254A201C1568002106
S11352F02E68042265E7C67F0097334001D0234817
S11353004BE7022120480A1CF2E636680424002EEA
S113531030D0281C0821032253E71A8A002A02D11C
S11353200598022303E03A8A0598291C0123FFF714
S1135330EBFC47E79A7C002A07D0114C1F2726680C
S1135340CC210136F05700F0F3FD0020011CFFF7DB
S113535019FD0EE00A4B1F20196801310856CB21B4
S113536005E007481F270468CA210134E05700F00C
S1135370DFFD0024201C2BB0F0BDC0461EF5FF1F2E
S113538020F5FF1F1CF5FF1F62B9000060B9000083
S11353902823044A5843136818180230C27F114363
S11353A0C177704720F5FF1F2822034B504319682B
S11353B008180430C07F704720F5FF1FF0B50D1C9E
S11353C02C352B7885B0061C0C1C9A070FD01121A4
S11353D0DA0700D41321FEF765FCC1B2002961D1BC
S11353E02F780326B743402007432F705AE0202725
S11353F01F4054D1088B002803D14024A3432B70B1
S11354004DE0CA681178A26A520516D504221342E7
S113541002D093432B7010E0221C2E32127801929A
S1135420914205D02D22125D8A4206D1012804D072
S113543004210B4301992B700127301CFEF732FC29
S11354402368402201332360287810432870002FFA
S113545028D1E56861690135E5608D4201D3A7680B
S1135460E760238B104A013B98B22083B6002F34A7
S1135470B5582778A98C002F14D0884212D86846D2
S113548000260123DD220273067246728772C372FC
S113549002A9301C052200F011FD267002E0301C28
S11354A0FEF7F6FB05B0F0BD30F5FF1F38B5051C5F
S11354B03020FFF7D1F8041E01D100240AE0281C93
S11354C0FFF7CAF8A0600028F7D043192061E06014
S11354D06361E583201C38BDF7B5019308AB061C56
S11354E00D1C141C1F78FDF7C7FD0198023808280D
S11354F000D9ECE004F090FA05486E3BC1EBEBEB0D
S11355009C0075483F010268D319E90401D59F68DE
S113551000E05F68002C28D0E20703D5301CFEF7BA
S11355204BFB04E0A30702D5301CFEF7A7FB610781
S113553003D5301CFEF7D4FA04E0220702D5301C50
S1135540FEF730FBBE6AE10603D580204201164314
S113555003E0A20602D561490E40BE62630604D58B
S11355607F243B1C25402F331D703D8DB0E05A4AEB
S11355703E0110685A4985196B689F6A0F4201D031
S11355801D8CA5E01D8BA3E0534A380111680F1848
S1135590BF68002D07D13D8BFE8B711B8DB2A142DC
S11355A000DB95E093E0FDF76FFD381C221C291CFD
S11355B0083000F0CEFB3C1C2C34051CFDF75CFDD0
S11355C0227860231A4200D082E0301C391CFFF795
S11355D0F5FE7DE040483A010368019299184F684E
S11355E0221C381C291C083000F0B3FCBB6A602460
S11355F0051C23426ED03A1C2C3211781020014233
S113560068D03C8BBF8CBC4264D88143117099062E
S113561060D5314B01991A68012350188168301CF8
S11356200C1C2C3427781F432770FFF7C7FE51E06A
S11356302948390102685618012C05D9023CB3687F
S1135640A4B2002D10D103E07368002D0CD107E043
S1135650012C05D976681D605D603560756037E0A2
S1135660A2000025D55033E0A4001F190020395CA6
S1135670295401300428FAD129E0174D3F01002CA8
S113568003D02968CF19BB681AE02B681024DA19F3
S11356905368191C2C310878204211D0A04308709B
S11356A091688B6A9A0608D50C1C2C342278012048
S11356B002432270301CFFF781FE2E68F5196B68D7
S11356C09C6800251C61DC601D831D8400E00025AE
S11356D0FDF7DAFC281CFEBD40F5FF1FFFEFFFFFBE
S11356E080800000F7B53B4E0091017A041C301C09
S11356F000F0A8F9051E03D0009A520705D467E00C
S1135700291C00F09FF9051E62D0334B6F1E1968E7
S113571038010F183E60009EB30707D5E088267A4B
S1135720FFF7C4FE2D4AB300D050B86000982C4E49
S1135730C30706D5A088FFF7B9FE217A78608B00ED
S1135740F050227A254990000B58002B0ED0226885
S11357509A62207A214B81005A58E088A17B0092FA
S11357604843642104F0BAF9009B9884207A8200AB
S1135770B158002926D0237B2F310B70207AA288C0
S11357808100607B7358504364210092019304F0BC
S1135790A5F9019A5084207A009A8100A07B73585D
S11357A050436421019304F099F901992268888493
S11357B0207A8300F1588A62237AA07A9900765875
S11357C02E363070227A211C3A73207AFEF72AF999
S11357D0281CFEBDD954000040F5FF1F30F5FF1F03
S11357E024F5FF1FF7B55B4A8B00061C9C585A48EA
S11357F080271D58A36A3F0101911F4014D0221C29
S11358002C32117804200F1C0740BC4603D081437E
S11358101170002710E0271C2E373F78B74202D1C1
S11358200143117094E067461A0605D5221C2D32F7
S113583011788F1B7A4257412020034218D0132E2F
S113584008D12E1C2C363378184330706868013028
S113585068607DE0112E0BD12F1C2C373978014262
S113586076D0814339700198291CFFF7A7FD6FE0BA
S1135870226801322260D9041AD5298BEB8B994214
S11358800CD8286906702A69696901322A618A423A
S113589001D3AB682B61288B013028832A1C2C325E
S11358A011786023194203D10198291CFFF786FD62
S11358B0208BE28B002F32D182420BD9013020831E
S11358C0206906702269676901322261BA4201D3F4
S11358D0A6682661A36A60210B421BD0261C2C36C5
S11358E03078C70616D4278B628C974212D3990658
S11358F009D52B1C2C331878022108431870291C55
S11359000198FFF75BFD357810273D4335706668D5
S113591001366660114BA26A1A4211D018E0258C38
S11359200135258482420BD92769013020833E70DA
S113593026696169013626618E4201D3A368236119
S11359402F342478002C03D060B20421FEF798FD94
S1135950F7BDC04624F5FF1F30F5FF1F808000000F
S113596008B5034B8200D158FFF728FD08BDC04697
S113597030F5FF1F13B5441E0548E4B20068230147
S1135980C318187B00941C680323A04716BDC046A7
S113599040F5FF1F08B5044B18700001FEF75CFECC
S11359A00249086008BDC0463CF5FF1F40F5FF1FD3
S11359B037B5031C0D1C0020FF2B0CD00648013BFF
S11359C00468DBB219016118087B00930C68022398
S11359D0111C2A1CA0473EBD40F5FF1F13B5441EF1
S11359E00548E4B200682301C318187B00941C68BE
S11359F00423A04716BDC04640F5FF1F13B5074951
S1135A00421ED4B208682301C218107B00210094FE
S1135A10146805230A1CA04716BDC04640F5FF1FA5
S1135A2013B50A1C0649441EE4B208682301C318CE
S1135A30187B00941C6800210623A04716BDC046AD
S1135A4040F5FF1F30B50A4B0A4A1B681478002240
S1135A50A2420BD01D680132854204D11D7B8D42C8
S1135A6001D1D0B203E0D2B21033F1E7002030BD4F
S1135A7040F5FF1F3CF5FF1FF0B5071C85B0101C57
S1135A80019102920393FFF7DDFF011E01D000256F
S1135A903AE0FFF7D7FF051EF9D01D4B461E1968E3
S1135AA03A8830010E18002A14D00398FEF7D4FD6A
S1135AB0041C70600ED038880090FEF7CDFD0028DD
S1135AC0E5D0009B6A46C11820606060A060108821
S1135AD0E160E0827C88002C11D00398FEF7BCFDC5
S1135AE0041CB0600BD07F88381CFEF7B5FD00287D
S1135AF0CDD0C31920606060A060E360E7826A468D
S1135B000299107931603073281C05B0F0BDC0468D
S1135B1040F5FF1F07B5032807D0052811D000283A
S1135B2013D1101CFFF7DEFD10E0938B01A80021B8
S1135B3012680380418011781823054AFFF79CFFFF
S1135B4004E0101CFFF784F800E000200EBDC046FE
S1135B50C55F0000F7B50E1C141CF10604D5202304
S1135B600421137001348E43F30706D5002804DAA8
S1135B7047422D202070013400E0071C00222C4DE8
S1135B800192002F34D0BD4213D9281C0A2103F0FE
S1135B9057FF019B051C002B03D10128F3D1B1074A
S1135BA001D5302102E07307EDD5202121700134A5
S1135BB0E9E7002D01D001210191291C381C03F0D3
S1135BC03FFF021CC0B26843303222703F1A0A21E0
S1135BD0281C03F035FF0134051CD2E7002F0CD03C
S1135BE0281C0A2103F02CFF30232370051C0134E8
S1135BF0019F002DF2D1002F0DD1651C710703D533
S1135C00202121702C1C06E03023B10701D523701C
S1135C102C1C23700134330704D50D200A22207074
S1135C206270023440273E4000D12670201CFEBD25
S1135C3000CA9A3BF7B50090C80602D5202313701A
S1135C40013248B2002804DA3024782514705570E3
S1135C50023240262027082307200F400B400E4025
S1135C600140CCB2BC460193042C00D90421C9B232
S1135C704D00EFB2141C3B1C013BDBB2FF2B10D0D8
S1135C8000989900C840051C0F210D403035392D6E
S1135C9004D960462735002800D0203D2570013402
S1135CA0EAE7D019019A002A04D00D270A240770C4
S1135CB044700230002E00D10670FEBD10B5031CE6
S1135CC01A78202A01D10133FAE700201C782F2CFE
S1135CD00CD90101201C3038C0B20133092803D982
S1135CE0201C57380F2210400843EFE710BD10B5B1
S1135CF0031C00221878011C3039092906D9002810
S1135D0014D02D2800D101220133F3E700201978A3
S1135D100C1C303C092C06D84400303CC00024182C
S1135D2060180133F3E7002A00D0404210BD00B5EB
S1135D308218031C934202D019700133FAE700BDA4
S1135D4010B50023934203D0CC5CC4540133F9E76B
S1135D5010BDF7B5041C151C0F1CFDF78DF9218A25
S1135D60628AE38A881846199E4202DD5D1AA91ADE
S1135D708DB2A068AA18E168628242190190A260FB
S1135D802E1C8A4205D32668D31A981B2A1AA360AC
S1135D9096B2FDF779F90198391C321CFFF7D0FF50
S1135DA0B54204D0B919AA1B2068FFF7C9FFFDF753
S1135DB063F9678AA18AAF4206D1228A0020AE180D
S1135DC077182782A08202E06B18A382781B608276
S1135DD0FDF75AF9281CFEBDF8B5041C0D1E33D17D
S1135DE00278407882425FD1FDF746F9A1782F4BC3
S1135DF02F481970FFF726FE2E49087000280DD091
S1135E002D4E013837680201B818436822791F8A79
S1135E10D88A7E1DB618864203DD0D70FDF734F96D
S1135E2042E006371F82A51DAC420BD09968277843
S1135E3001340F70DA68013199609142F4D31E681D
S1135E409E60F1E706252FE01A4B1E78002E0CD138
S1135E5001784378994226D187781548391CFFF791
S1135E60F1FDFFB2061E06D11DE0104A002017788E
S1135E701870FDF709F9104A013E10683101E678FF
S1135E8043185868032E04D1C58A048A2F1BBDB257
S1135E900AE0211C2A1CFFF75CFF0421051C78B2D0
S1135EA0FEF7EEFA00E0351C281CF8BD3EF5FF1F96
S1135EB0C55F00003DF5FF1F40F5FF1F08B5031E39
S1135EC004D1081C111CFFF787FF05E00020FF2BFD
S1135ED002D0181CFFF74EFD08BD38B5041C031C86
S1135EE01D781A1B92B20133002DF9D1281C002A07
S1135EF003D0081C211CFFF7E1FF38BD08B5024B95
S1135F001978FFF7EAFF08BDE6F0FF1F1FB56A46E0
S1135F10FFF790FE6846FFF7F1FF05B000BD1FB51F
S1135F206A46FFF717FE6846FFF7E8FF05B000BDB5
S1135F3007B5031C002083420AD06A4610705070D3
S1135F400120D0701171684605219370FFF744FF5A
S1135F500EBDF7B5038A041C0E1C4768151C9A4233
S1135F6000D91D1CADB2002D28D0E0687A196260FA
S1135F70824215D3C11B8BB22268E81A11186160E2
S1135F8000930190FDF780F8002E12D0391C009A7E
S1135F90301CFFF7D5FE009F2168F019019A06E036
S1135FA0FDF772F8002E04D0301C391C2A1CFFF7B0
S1135FB0C7FEFDF761F8268A731B2382FDF764F898
S1135FC0281CFEBDF8B51D1C06AB0F1C161C1C7846
S1135FD0FDF752F8052D0ED0062D13D0042D1CD13B
S1135FE01048220101688D186868391C321CFFF7BB
S1135FF0B0FF071C14E00B4A26011568AB195C6856
S1136000278A0BE0074E240133681F19786800279C
S1136010016807828160416000E00027FDF734F8E1
S1136020381CF8BD40F5FF1F30B50023934206D05D
S1136030C55CCC5C0133A542F8D0012000E000200F
S113604030BD00B50378002B0CD00A78934206D0FB
S113605000209A42404140420121084306E00130B9
S11360600131EFE7087843425841013800BD00B5DB
S11360700B78421C03700B780131002B01D0101CEB
S1136080F6E700BD00B5021C031C1978981A013309
S11360900029FAD100BD0000064B0A0E18705A7090
S11360A0080C0A0A197100219870DA70181C5971C9
S11360B07047C0464CF5FF1F10B51849FF230B70FD
S11360C00B1C174A147864B2002CFADA0978FF29F9
S11360D0F3D0FE291ED18024A1004118FF241C7096
S11360E0147864B2002CFBDA1C7804700130884206
S11360F0F4D10A49FF200870147860B20028FBDA52
S11361001978FF211970147860B20028FBDA1B7823
S1136110002001E00423584210BDC0460670074029
S11361200070074010B5021C031C0B3200201C78C1
S1136130C1014008201841180133C8B29342F6D176
S113614010BD000000B50B4A81239800115C0029A2
S113615005D009490020535C834209D101218801FB
S11361604318D900501880229300C11801220A71E3
S113617000BDC04658F5FF1F0C04000010B51F49B0
S1136180FF230B700B1C1E4A147864B2002CFADA3D
S11361900978FF29F3D11949FE240C70147861B2EF
S11361A00029FBDA80241978A10041180478013011
S11361B01C70147864B2002CFBDA1C788842F5D188
S11361C00E49FF200870147860B20028FBDA1978B1
S11361D0FF211970147860B20028FBDA1978FF21C6
S11361E01970147860B20028FBDA1A781F23134060
S11361F00020052B01D00521484210BD0670074040
S113620000700740044B08211A8B32200A431A837A
S1136210024B18607047C046D8F9FF1F74FBFF1F7C
S113622010B50A4C201C216800F01AF900280CD182
S11362306369FF2251005C5C552C02D0032040426C
S113624003E0034A9B5CAA2BF8D110BDD8F9FF1FC9
S1136250FF01000038B50E490E4B1022041C01202A
S11362601A60086002224D206421FEF73FF90A4DAE
S1136270002C03D08024A100298307E00748FFF7FE
S11362803DFE8022064853002B83046038BDC0467F
S113629074FBFF1FC4F00F40D8F9FF1F70B9000052
S11362A040FAFF1FF7B5434D161C434B2A68071CE1
S11362B00191424C9A4205DD4148FFF71FFE02203E
S11362C0464260E02068002802D006285AD127E020
S11362D01522013A002A62D03A4BFF2119703A483C
S11362E0017849B20029FADA1B78FF2BF1D1226830
S11362F0052A0CDCBB5C33490B70027853B2002BCB
S1136300FBDA22682F4901320B782260EFE7286814
S1136310002805D000214D20FEF7B2F800212960A5
S113632023685A1C22601A2B05DD296806220131D4
S11363302960226036E0234BFF2018701A1C224982
S1136340087840B20028FADA1B78019803705BB22F
S1136350002BE5DB002E15D03F780423492F00D114
S1136360122300272760206898420BDAFF27177052
S1136370087847B2002FFBDA1078276830700137AD
S11363800136EFE700262F68002F05D04D200021AD
S1136390FEF776F800232B600021216008E02C68CA
S11363A001342C604D200121FEF76AF801256E426C
S11363B0301CFEBD74F9FF1F204E000034FAFF1F8D
S11363C089B900000670074000700740F7B51E4DFC
S11363D00E1C2B680421194003D00024042931D158
S11363E00BE0008B400600D45202184F04210B43EB
S11363F010243C602B60164B1A60154A6F461168D6
S113640058200737FFF748FE391C0022FFF74AFFE0
S1136410041C10480460002C14D1397800290AD1D6
S1136420301CFFF7ABFE002805D00B480525FFF70D
S113643065FD6C4206E02A68084B04271026BA431F
S11364401E602A60201CFEBD40FAFF1FC8F00F40EA
S113645030FAFF1F3CFAFF1F96B90000C4F00F404A
S1136460F7B5244C02222368051C1A4002D0022AE4
S11364703DD10BE0008B400600D449021E4F02229E
S1136480134310263E6023601C4B19601B4F5120A0
S11364903968FFF701FE694607310022FFF702FF62
S11364A017490860431CF1D0164E00280ADB6846E1
S11364B0C279002A15D16869FFF7FEFD104B1860F8
S11364C0002806D0256802271022BD4332602560CB
S11364D00EE0298B480602D43868420A3A603F68C5
S11364E02F602368102535600226B3432360002003
S11364F0FEBDC04640FAFF1FC8F00F406CF9FF1FF5
S113650078FBFF1FC4F00F40F7B5224E0422336816
S1136510051C1A4003D00024042A38D10BE0008B58
S1136520400600D449021C4F0422134310243C604B
S113653033601A4B1960194F58203968FFF7ACFDC6
S1136540694607310022FFF7ADFE1549041C0860B7
S11365501DD16846C279002A12D16869FFF70EFE80
S1136560002805D00F480526FFF7C8FC74420EE04A
S11365702B8B580602D43968480A38603F682F606C
S11365803168094A04231025994315603160201CA1
S1136590FEBDC04640FAFF1FC8F00F4070F9FF1F50
S11365A07CFBFF1F96B90000C4F00F40026838B5A9
S11365B0041C0D1C8A4212D0038BDA0709D5201C57
S11365C02168FFF7A1FF0130F9D0208B0121884316
S11365D020832560201C291CFFF742FF00E00020D7
S11365E038BD0000F0B51F4C85B02368019202222B
S11365F01A401D4D02D0022A31D10BE0008B400617
S113660000D44902194F0222134310263E6023602E
S1136610174B196016496F46096851200F37FFF769
S11366203BFD391C0022FFF73DFE2860421CF1D0DF
S1136630104E002806DA2268102535600226B2437F
S113664022600DE03878002803D10198FFF734FD6B
S1136650286021680223102299433260216028684F
S113666005B0F0BD40FAFF1F54F5FF1FC8F00F40FE
S11366702CFAFF1FC4F00F40F0B5171C54225143ED
S1136680464B474CA5445C18A168251C2B35401A81
S1136690297803F0D5F96668236A8019C2097F2135
S11366A0D51808400390291C201C04AAFFF79AFF60
S11366B000260196B04217D00425684269E0666856
S11366C0B3421BD9022F3CD1364F10326E4697513C
S11366D00F1C206AD9097F260A18334002920393BB
S11366E0029B0026AB423ED10398102382006946E8
S11366F09E187358002118011030E0D1022F47D0A2
S1136700002304A98B50208B410707D5276B019ADE
S113671001370223BE181843266320830026301C49
S1136720211C2A310F78B74233D9E06904A9704398
S11367304219201CFFF74AFE411CF6D00136F6B27E
S1136740EEE7103268461150019A01320192C0E717
S1136750E269201C724304A95219FFF737FE013085
S1136760F6D00136F6B2211C2A310878B042EFD8AF
S1136770201C04A92A1CFFF729FE0130F8D0201C94
S1136780029904AAFFF72EFF002895D1029DABE7DA
S113679000208524A400A544F0BDC046D8F9FF1FFD
S11367A0ECFDFFFFFFFFFF0FF7B50E1C8121071C57
S11367B001938800135C0225141C1D4029D0156820
S11367C0B26B954238D05A070CD5211D381C22686B
S11367D0FFF7FCFD0130F8D081208300E55C042143
S11367E08D43E554019A002A0CD1221D381CB16B4B
S11367F0FFF7F8FE002802D0042465421DE0B56BC3
S1136800256019E08127BE00A05D02239843A055AE
S113681012E0019A002A10D1221D381CB16BFFF737
S1136820E1FE0028E8D1B76B8126B0002760235C25
S113683002210B43235400E00025281CFEBD000068
S1136840F7B5161C02681D1C08AB1F888A4206D1C6
S113685044693A1C6119301CFFF772FA7FE0414C1D
S1136860022223681A4002D0022A78D10BE0008B5E
S1136870400600D449023C4A102010600220034321
S113688023603A4B1960394951200968FFF704FC29
S1136890694600220731FFF705FD354A1060421CA6
S11368A0F1D0002807DA25683249022310229D43DB
S11368B00A60256054E06846C379002B48D12E4A0B
S11368C0FF211170131C2D49087840B20028FADA10
S11368D01078FF28F3D00022FE2808D02848FFF7BC
S11368E00DFB35E0087840B20028FBDA1878AA429C
S11368F004D0FF200132187092B2F3E72A1C7819F1
S113690080B2824210D2FF200132187092B208780D
S113691040B20028FBDA187830700136EFE70F78C0
S113692078B20028FBDA1878164DFF261E70AA42AA
S113693002D8013292B2F2E70F787AB2002AFBDA77
S1136940FF201A7818700E7875B2002DFBDA1B78C8
S11369502668084B02251021AE43196026600020EA
S1136960FEBDC04640FAFF1FC8F00F407CF9FF1F70
S113697044F5FF1FC4F00F40067007400070074045
S1136980A4B90000FF01000030B50B68026A041CC2
S11369900D1C7F20D90985B0034089180422009278
S11369A09B00201C03AAFFF74BFF00280FD1039B79
S11369B061688B420DD9626A93420AD8211C2B600C
S11369C02B310A78E46853431B196B6003E00425F8
S11369D000E00725684205B030BD70B50B7A051C90
S11369E00133D8B208722A8D0C1C00265109884242
S11369F011D3606826720130AB682A1C60602B32A8
S1136A00C01A117803F060F8B14204D1281C211C8B
S1136A10FFF7BAFF061C301C70BDF0B54B6A161C9C
S1136A20026887B0041C0192002B31D003AD2031E1
S1136A30281C0C22FFF784F900203070218B0127D9
S1136A4039432183201C6968FFF7B0FD002821D158
S1136A502A7A60695301C318E5211A7819703078CD
S1136A604021C31933708A43BA4204DD201C291C17
S1136A70FFF7B3FFE2E7268B3E4209D0201C0199C1
S1136A80FFF742FD0130F9D0258B0127BD43258353
S1136A90002001E00424604207B0F0BDF0B5456871
S1136AA091B00B1C05910B9206953A330768041CB0
S1136AB01878542250438D490C220E18291C0DA815
S1136AC00896FFF73DF93D785C2D01D02F2D00D1BC
S1136AD0013700230A93201C1E3020210B22E76279
S1136AE00490FFF724F9211C2931182200200A7090
S1136AF03D1C0790021C01213B7801370D2B13D05C
S1136B0004D8002B14D00A2B15D10DE02F2B0FD055
S1136B105C2B0DD02E2B0ED1002A7BD0082A5EDCF4
S1136B20012008223D1CE7E7002A79D02F1C7BE0D6
S1136B30002AF7D0FAE7202B04D8002AF2D0202B21
S1136B40F0D14AE07E2B34D8694EF518213D2D78DA
S1136B502126354207D0079E002E01D0AE063ED432
S1136B606B063AD4DEE7079E002E38D16E070DD5AA
S1136B70049EF57A012804D00826B543049EF572D4
S1136B802DE01026B543049EF57241E008263542F7
S1136B9025D0049D203BDBB2E97A012803D00E43C3
S1136BA0EE7203211BE01026049D3143E972032198
S1136BB02EE01E1C7F36F5B21E2D04D91E1C203675
S1136BC0F5B21C2DAED8002A09D1E52B22D1049AA6
S1136BD00523137001220792A4E75F230421072AE7
S1136BE018DD002809D00A2A14DD06E00D2A09D888
S1136BF0002A18D00A2A16D0071C3A78781C0D2AC5
S1136C00F4D110E02F2A01D05C2AF5D102210BE047
S1136C10072AE8DC049D0026AB540796013281E77D
S1136C200123594200E00421A161013100D17CE13A
S1136C30676327633E785C2E01D02F2E00D1013785
S1136C4000220992069908984D68291C0295FFF7BD
S1136C50ADFC061E00D063E1069A0898117A4369D8
S1136C6009984D015D19002833D10A9800281AD1DA
S1136C70261C3836111C301C0C22FFF761F80B9BC4
S1136C802878002B02D1E52834D1A6E1002831D0A0
S1136C90297B00292ED1AA7E002A2BD1EB7E002B42
S1136CA028D10B9B2DE00A9B013B0A93002B00D0BB
S1136CB022E1216D132900D9A1E10D264E4351365D
S1136CC04A1CFF362265A019291C0B22FFF738F84D
S1136CD012E1281CFFF726FA95239A00A15C099675
S1136CE0814252D10126A66109964EE0D8F9FF1FD0
S1136CF013BC0000E97A3F220A400F2A00D0C8E002
S1136D0000230793420601D5606B20630D22013AEC
S1136D1000D312E12978490600D450E1201C311C2B
S1136D200C224430FFF70CF895266A7BB300E2543A
S1136D3028783F230340226BE16A012B00D047E10E
S1136D40012676428A4200D0BAE0606B1E1C2063A2
S1136D50AE4BE05C00280CD00138C1B20C22E154E7
S1136D60514360316018211C5431FEF7E9FF0022C1
S1136D70A265A64800232354B21C00D1D2E0012E00
S1136D8000D13FE1033600D0B6E0A669012E02D05F
S1136D90032E00D0B0E02B78002B02D0E52B11D1CC
S1136DA0AAE06769390700D4ADE0059D01222E8F62
S1136DB0181CEB862B6832402A87002B00D1A2E0F6
S1136DC01870A0E0099900291ED0012009906E7D59
S1136DD02B7D3106EE7E1A048818AA7E31024318F0
S1136DE0059E9818E0607560ED7A10231D4216D157
S1136DF0059D089AE8622B321678089B7043D9687F
S1136E00401828630220FFE0EA7A110774D4281C92
S1136E1004990B22FFF708F90028D8D06CE0A16987
S1136E20002904D0A28B1A4201D00020ECE0069D78
S1136E30089E28602B36337808995843CA6802267E
S1136E40801868602E723D78002D15D16469032086
S1136E50022C00D1D8E02107E7D5059F0598143707
S1136E60391C0C220830FEF76BFF0598391C0C22E4
S1136E702030FEF765FFD8E70DA806990C22FEF72F
S1136E805FFF099B2760002B00D124E60421A16148
S1136E9021E6032600284BD07642082900D1A0E041
S1136EA0236D00200790132B0AD80D225A43513228
S1136EB0591CFF322165A018291C0B22FEF740FF44
S1136EC0636B079900202363A064002900D18EE03E
S1136ED0321D00D03CE74D4D625D002A05D1201CD7
S1136EE0543006990C22FEF72BFF665D132E00D951
S1136EF085E046480136265408980699FFF76DFD4B
S1136F00002800D19EE6A769002F0ED0A48B21078C
S1136F1004D506980DA90C22FEF712FF062605E0FB
S1136F20042603E03D78002DF8D0032670426BE080
S1136F300526082AB0D00226AEE7501E0B281FD81B
S1136F4002F06AFD1C1A18161412100E0C0A080618
S1136F50AB7F16E02B7F14E02B7E12E0AB7D10E0BC
S1136F602B7D0EE0AB7C0CE02B7C0AE0AB7B08E0D5
S1136F706B7A06E0EB7904E06B7902E0EB7800E0F1
S1136F806B78FF2B00D1C2E6002B00D1BFE6216B4A
S1136F900139216309788B4200D1B8E6181C4138C5
S1136FA0192802D82033DBB205E0181C61381928EF
S1136FB01AD82031C9B28B4200D1A8E614E0952634
S1136FC0B300E05C697B161C884200D078E7AFE62A
S1136FD000268A4200D3BBE606E00B9E04220796F5
S1136FE003E0002307936BE70122564268E7711C14
S1136FF000D06DE729783F2211400A91A8E60023CA
S11370000A9379E7099677E711B0F0BD55020000BD
S1137010F0B589B002900D1C141C0393002801D014
S1137020984800E09848FEF769FF281CFEF766FFC1
S1137030626A002A03D19548FEF760FF71E0944824
S1137040FEF75CFF9348FEF759FF231C283318789A
S11370508121FEF75BFF9048FEF750FF8421606AB0
S1137060FEF754FF8D48FEF749FF8421206AFEF79E
S11370704DFF8B48FEF742FF206854263A300178D2
S1137080884F71437F18211C203105A80C2200254C
S1137090FEF756FE0095381C0699FFF787FA05AEF1
S11370A0019000283DD1327A7B695001009A1E1864
S11370B03178002A12D1402319420BD00D1C9D4374
S11370C07948FEF71BFF0821281CFEF728FF012141
S11370D000910DE07548FEF711FF09E0013D012024
S11370E0EDB200908D4203D07148FEF707FF019D79
S11370F07048FEF703FF321C203201923078912150
S1137100FEF704FF019801368642F7D16A48FEF77C
S1137110F5FE012D05D0381C05A9FFF75EFC0730EC
S1137120B9D16648FEF7EAFE8121207FFEF7EEFE24
S11371305948FEF7E3FE8421A069FEF7E7FE574FA6
S11371405425381CFEF7DAFE84216069FEF7DEFE62
S11371505348FEF7D3FE266852493A3633785D43E6
S11371604D19281CA169FFF721FA002800D087E0F7
S1137170227F6F6950013F183E1C20364D48FEF7B0
S1137180BDFE00963E1C30789121FEF7BFFE009BA9
S113719001369E42F7D14A48FEF7B0FEF97A042937
S11371A010D005D801290BD0022911D1454810E08F
S11371B0102909D0202909D0082909D1424808E01A
S11371C0424806E0424804E0424802E0424800E007
S11371D04248FEF793FE4248FEF790FE0026BA5D51
S11371E005A8131C203B5E2B00D92E2282550136A4
S11371F00B2EF4D10027C772FEF780FE606A0028C8
S113720009D03848FEF77AFE9521039B8E00985DDD
S11372108121FEF77BFE029A002A09D03248FEF74C
S11372206DFEA0680021FEF77AFEE76A246B07E092
S1137230039C281C2B30E7680178EE6879438C198D
S11372402D6AFA0929485619FEF758FE8421201C94
S1137250FEF75CFE1148FEF751FE8421381CFEF750
S113726055FE2348FEF74AFE8421301CFEF74EFEED
S11372702048FEF743FE7F2038408921FEF746FE72
S113728009B0F0BDAFB90000B6B90000C2B9000042
S1137290CCB90000D5B90000BFBA0000EAB90000BB
S11372A046A90000D8F9FF1FF5B9000008BA00008C
S11372B01DBA000030BA0000ACB9000037BA0000B3
S11372C052BA000069BA000077BA00005FBA000041
S11372D070BA000081BA00008BBA00000FB9000038
S11372E093BA000098BA0000A5BA0000B6BA00002C
S11372F0CBBA0000D9BA000010B50B0A8176C37668
S11373000B0C090E041C03754175C2720021042282
S11373101C30FEF70CFD632243236620B421A075C4
S1137320E1752276A2746376E374A073E173227428
S1137330637410BDF0B5964C036AA5440192041C15
S113734001980C220F1C104207D1218B490703D549
S1137350676B256BAF4200D96768FE09F2187F237B
S11373603B40059369461420455C069202950492BD
S11373703D1C201C04990CAAFFF734F9002800D006
S113738000E1029E0CABB200D158002900D0E6E027
S1137390019A910710D1029F7E4ABE00019B3036AC
S11373A068463250590700D497E0059900228F00AF
S11373B030373D50019290E0231C2B331978E0685C
S11373C0099169430E180796079B7202089203936A
S11373D009990798039A0E18B31AD9B20029DAD07A
S11373E0231C2B331878884241D10199C9073ED513
S11373F08CAE80239A00301C0021FEF798FC301CD0
S113740020210B22FEF793FC2E223270301C391CF3
S11374101022FFF771FF20210B2294A8FEF787FCAE
S11374205D4E5E492E2069446E44C8771022F07781
S1137430022194A8FFF760FF201C8CA9039AFEF791
S1137440C5FF0130F8D03FE0042B3DD1544B6E46CC
S1137450196858202F36FEF71FFE311C0022FEF754
S113746021FF50490860002815D001302CD14E4A24
S1137470042316683340E7D1208B089B400600D5CF
S1137480039B4A4910220A600420474A06431660B7
S1137490434E3360DAE7317800290DD180228CA87D
S11374A09200FEF744FC8CA8FEF768FE002803D087
S11374B03F48FEF723FD07E03B4E3E4B3168042274
S11374C01020914318603160039B089A8021880042
S11374D001331618039308967AE70026271C2A37E7
S11374E03878B0420CD9E169049A7143201C8A1897
S11374F00CA9FEF76BFF0130F5D00136F6B2EDE7CB
S1137500019B190703D4278B7A071CD43CE0201C69
S113751006990CAAFFF766F8002833D105990CAA3E
S11375208E00B550061C3878B042ECD9E369069851
S113753073430CA91A18201CFEF748FF0130F5D03C
S11375400136F6B2EFE7636B9D4201D3691C6163B8
S1137550226B02263743013A2783226314E0029800
S113756001357F2804D0061C0136F2B2029208E7E6
S11375700199049804239943013000260191049051
S11375800296F6E604256D42281C0B4CA544F0BD7A
S1137590CCFBFFFFFFFFFF0F3202000031020000AF
S11375A0D4F9FF1F48F5FF1F40FAFF1FC8F00F4032
S11375B096B90000C4F00F40340400007FB50B6896
S11375C0041C006ADE090D1C3618002A0DD12A6835
S11375D07F21114004208B000090311C201C03AA41
S11375E0FFF72EF9002824D106E0201C311CFEF7F9
S11375F0DDFF00281DD1EAE7039B6668B34202D988
S11376000E498B4205D9201C29680C22FFF792FEF3
S113761003902B68626A072093420BD80398261CB8
S113762028602B363178E468484303196B600020E6
S113763001E00420404204B070BDC046FEFFFF0FCD
S113764070B5047F4B69061C60010D1C1C18081CD6
S1137650B169FEF7ABFF00281DD1B1680A0A080C16
S11376600B0E21776277A077E377632043236621AB
S1137670B422A175E2752076A0746376E374281CA5
S1137680B169FEF741FF0130F9D02E8B0124A643E6
S11376902E83002001E00425684270BD71B5C56ADF
S11376A0FFB0291C6A46041CFEF79CFF002802D088
S11376B00424604229E0206BF42256006946144AEF
S11376C088556E46010AB154F522010C5200B1549A
S11376D01049636B000EF622705450000E4A190ACA
S11376E0B154F72133544A00180CB0540B481B0E04
S11376F03354201C69462A1CFEF768FE0130F8D07A
S1137700258B0226B543258300207FB072BDC04679
S1137710E9010000EB010000ED010000EF010000B1
S1137720F0B593B00791D90F08900D920E930A917A
S11377304668846805D0B94B0799C218201CFFF726
S11377406CF908988269022A07DC201C7168FEF72C
S11377502DFF051E00D169E1CBE10D98FEF792FCE7
S11377600D9F089B39181E3305900B910C220021A4
S1137770181C0993FEF7DBFA089A2020171C073718
S11377802F219077F977FCF7DDFD071CFCF7DAFD74
S11377900304A3481F4307401197F4D0089811A984
S11377A004222030FEF7CCFAFCF7CCFD9D4A11A947
S11377B010401190089802222430FEF7C1FA09986B
S11377C0FEF7B0FC05990F90013109910127099B3F
S11377D00D2B05DD099B01370D3BFFB20993F6E73D
S11377E03B1C132B13DC0C22101C584308998446B1
S11377F0081C6044416E002907D06046089B603035
S11378001918301CFEF79CFA01E00133E9E7201C4B
S11378107168FEF7CBFE002800D06CE1327A616912
S1137820500140220B183A430120FF2706930C9283
S11378300597404209990D2903D10B9F3B780027F6
S11378400593431E0130202800D9D6E002F0E4F865
S11378505A11747D7F84868B8D929499D5D5D59B4E
S1137860A1A3A8AAAFB1B6B8BDBFC4D5D5C6CCCE66
S1137870D300311C201CFFF7B0F8C11D2ED1756850
S11378803368206A013D7F227560D90904251340BD
S113789009189B000095201C11AAFEF7D1FF0028AF
S11378A000D028E1119B61688B4202D95E48834273
S11378B005D9201C31680E22FFF73CFD1190326877
S11378C0656AAA4200D916E1119B211C33602B3151
S11378D00878E26843439D18756002E0002800D0F0
S11378E009E1201C7168FEF761FE002800D002E166
S11378F0337A606959010B9D0D9B421806929D4293
S113790000D285E0002120220698FEF710FA0C9D93
S11379100CAB40221978069895432B1C0F2201705A
S1137920013BC2720FA8D9B20578069B0C915D7316
S11379301D1C1F23181C7DE768461422115C0122BC
S11379406970208B1043208357E0AF70F2E76846DC
S11379501422115CE97050E02F71EBE768461422A1
S1137960115C697149E0AF71E4E768461422115C67
S1137970E97142E02F72DDE768461422115C6972F6
S11379803BE0AF72D6E714236846195C0A23A97357
S113799033E0EF73CEE7684614210A5C2A742CE0C6
S11379A06F74C7E7684614210A5CAA7425E0EF7473
S11379B0C0E7684614210A5C2A751EE06F75B9E7B2
S11379C0684614210A5CAA7517E0EF75B2E76946A8
S11379D01420425C2A7610E06F76ABE714236846E5
S11379E01A5C19232A7708E06F77A3E76846142204
S11379F0115CA97701E0EF779CE709990D2903D180
S1137A000B9801380B9095E7099A0132099291E796
S1137A10069F002F00D098E66DE0C0465602000095
S1137A201F1F1F1F1F1F0000FEFFFF0F317A626917
S1137A304801089917181E31381C0B22FEF780F9EB
S1137A40089B0A98293319783973002816D1079DA1
S1137A50201C002D08D131680122FFF76BFC051CA6
S1137A60291C381C102207E00A990A1CFFF762FC43
S1137A70051C291C381C2022FFF73EFC201C7168C1
S1137A80FEF742FD0130F9D0268B012296430A9F6E
S1137A9026830026B74225D1079BB34222D019681A
S1137AA0181C20310C221430FEF74AF90799201CC7
S1137AB0CD622B300278E7685543081CED190D633D
S1137AC008222C313430FEF73BF907990E9B8E6067
S1137AD0CE600E684B60301C3A3002780F1C3E3783
S1137AE03A700226258BA90707D5201CFFF7D6FD7F
S1137AF003E0042700E007277E42301C13B0F0BDEA
S1137B0073B5061C0C1C151E08D16A46201C311CBA
S1137B100732FEF782FF002813D030E0036800220A
S1137B2058686621027742778277C277817563222B
S1137B304321B423C375027682744176C174022D45
S1137B40E3D1201C2168FEF7DFFC0130F9D0208B43
S1137B50012398432083306BA668B04207D2208B60
S1137B60022528400BD0201CFFF798FD07E0221CBB
S1137B70483211782A1CFEF77FFD0028EFDA76BD23
S1137B80F0B5C94CC94DA5446E462B682736002173
S1137B9007903170980707D5C548FEF761FC011CB2
S1137BA0421C01D100F090FD2A68D30701D500F0F2
S1137BB006FDC04C2068242801D900F05EFD01F0C8
S1137BC035FF25002500650078008C00AA00B80068
S1137BD0C7005C055C05E0005C055C055C055C05B4
S1137BE036014201B30166025C05E202220300048D
S1137BF00A04360456045F045C055C055C055C05F8
S1137C0075045C05A004EC045C05CF02AA4F802631
S1137C1039683204A94B0A433A60186880256F0119
S1137C208026A7493843B20018600A601868902576
S1137C30A44A3843AE00186016601968A248A34DE0
S1137C403943196028601E68032037431F60A04F22
S1137C5010214022FCF74CFA3A6810231A439D483D
S1137C603A6001689C4E19435C259C4A0160732765
S1137C7035709B489B499C4D177002780A782B609D
S1137C800121022323604D200A1C79E20B27013FC6
S1137C90002F09D0934AFF211170914B187845B2F7
S1137CA0002DFADA1278F2E7904B102103201960C4
S1137CB020608F48311C0022FEF7F4FA002805D01A
S1137CC0013001D100F000FD002535703278012A21
S1137CD001D000201BE0042727608648311C0CAA31
S1137CE0FEF7E0FA002854D13678012E0BD1332167
S1137CF069440B78AA2BECD1322068440578012D15
S1137D0021D07D4800E07D48FEF7F8F80120FEF719
S1137D10A1FA00F0B2FC7A48311C0022FEF7C2FA44
S1137D20002836D13778012F01D900F0C3FC062290
S1137D3022607448311C0022FEF7B4FA002828D1CE
S1137D403178002902D0052700F037FC072525608B
S1137D500CAF6D48311C3A1CFEF7A4FA002818D168
S1137D606A48FEF7CBF8387840221040504B02D0D6
S1137D701A83674801E018836648FEF7BFF80A21B2
S1137D8021600CAD6448311C2A1CFEF78BFA0028D4
S1137D9003D001309DD100F097FC454E6946301C5C
S1137DA0323138301022FDF7CBFFAF78687AA97AE8
S1137DB07A0608D5ED7A03040902581842190132EB
S1137DC09702376118E02B7A032213409F02800048
S1137DD03B188909E87A5F182B7B02405200D909C5
S1137DE050180137023087403761ED790F222A405D
S1137DF00A2A01D17F0037614848FEF77FF873698A
S1137E00002B04D180218800FCF726FC70610F2030
S1137E10206004214D20FCF733FB48360024324D0A
S1137E202E4A347010262E60147000F026FC204870
S1137E3000270760FEF7F4F9011C451C01D100F08E
S1137E4043FC10262660CF1C00D1DDE01122226005
S1137E50002900D03DE7164CE123656959006F5CA9
S1137E60261C002F1CD0281C52300278462A17D01A
S1137E702B4BE426E95C70000F062A492A5C6E5CF1
S1137E801304FF183002E3233A185F00ED5D511923
S1137E902160FEF7C5F9011C481C45D100F014FC13
S1137EA00024346042E0C046CCFDFFFF40FAFF1FCF
S1137EB0D8F9FF1F74FBFF1F34800440388004404E
S1137EC014C0044018C00440030200001CC0044055
S1137ED0C0F00F40D4F00F4003700740017007401A
S1137EE00070074006700740C4F00F40C8F00F4010
S1137EF001BC00006AB90000E2BA0000FABA00004E
S1137F0077BC00000DBC000071BC00001FBB00006A
S1137F102DBB00003DBB000007BC0000ACB9000055
S1137F20C9010000C701000003316DD0DB4B0025FF
S1137F305C69E07DA77D267B0202D219310204959B
S1137F40AA4210D1261C0836F07FE21DD57F070611
S1137F50A01DC27F2E04BF1915027E19671DF87F6C
S1137F60012532180495267DE07C37023D180195E1
S1137F70002D0ED1261DE01CF77FC67FA01C3D06F8
S1137F803704C67F601CED193702C67FED19AF199F
S1137F900197DA61277C1D1C2A352F70667B1D68CA
S1137FA0181C2B3005950670E07B0502A07B2D186C
S1137FB0A8B2059D03904019B94D06901862A942D4
S1137FC007D9002E05D00D1C754380200002854280
S1137FD001DDB44816E0574302971A8B0825202088
S1137FE0AA4302431A831985039BD919019F781A5E
S1137FF0311C01F025FDAC4A904208D8049D002DA7
S113800005D1AA48FDF77AFFFEF7FCF835E3201CFA
S11380103130271C037830373A78201C19022F306E
S11380208D180178013802780F06211CABB22D316E
S1138030150478190F783A028518201C2C30017821
S1138040059A6F18954D9B1801980399EB622B6064
S1138050029B421AD01A311C6F6001F0F1FC7E437E
S11380600699686202984218961B211C281C473105
S1138070AA60EE600B224930FDF762FE8C4F122499
S11380803C60FEF7CDF8011C421C00D11CE3834E7A
S1138090002952D1328B53044FD47369804D585DFB
S11380A0AA284AD1FF214C001F5D552F45D1DD7808
S11380B0412D42D1987861283FD1597852293CD139
S11380C01C78522C39D17B4FDD5D612D35D1F320E5
S11380D041005C5C412C30D1774FDD5D722D2CD199
S11380E0F22041005C5C722C27D1744FF5214C00C6
S11380F0DD5D1F5D28063D04411971481C5C2702A3
S1138100CD19F42148001C5CF7202F196D4D3763FD
S1138110595D45000C06595D6B4D0804595DF62503
S11381202418080269005B5C2418E018023F70639D
S1138130B84202D804273A4332836448FDF7DEFE8E
S1138140348B8022144334836148FDF7D7FE614E9B
S113815001213568564B29431320316018600CE027
S11381604E480168FEF77CF9002800D0B1E52A6882
S1138170012013261043266028604D20C8210422C4
S1138180FCF7B4F979E2454F80227D690021920021
S1138190281C3E69FDF7CBFD4F4B0220E022E8543A
S11381A00C215000E12329545A000B21A9544B49B6
S11381B03820E2236854F82258002A54484AB82147
S11381C0E3233F3EA9543F205900E522454B685420
S11381D05000310A2E54E954E620434B320C41003E
S11381E0360E6A54FF20EE542D4B41005522AA2628
S11381F06A54EE54381C0021FEF786F9002800D09A
S1138200D1E115272760254DFE226C69520000211B
S11382109026201CFDF78BFDEB205821A670E61C50
S113822020706170301C3149FDF721FF80239F00CD
S11382302F85002202273F20E272277320762077C1
S11382402869F8236375031C3F3B621CD3772774AA
S1138250A21C1F0AD7771F0CF777FF211E0E221DC1
S1138260D677A1762F1C20218226A1732B373203C7
S1138270934201D801233CE080267204934201D842
S1138280082336E08026B204934201D8102330E05C
S11382908026F20493422BD839702BE0D8F9FF1FC3
S11382A0FF01000048BB0000F4FF000055BB0000C4
S11382B074FBFF1FE7010000E5010000EB01000073
S11382C0E9010000EF010000ED01000061BB0000C6
S11382D0ACB9000040FAFF1FBF010000C301000059
S11382E0C5010000CB010000CD01000070BB0000FF
S11382F040233B702F1C2B3739786038C90101317A
S1138300401801F09DFBC34E621D010AA31DD077E6
S11383103060D977060CE11D020E4000CE775F3045
S11383200131CA770223243101260622A860201CC9
S11383300B700E718A715230B7490822FDF700FDA7
S11383403F78AB6879005A1AEA60261C6773271CC9
S1138350292180204237403639703070FBF7F2FF14
S1138360231C43331870FBF7EDFF221C44321070BA
S1138370FBF7E8FF271C45373870FBF7E3FF211CA8
S113838046310870281C49300278201C00244730EC
S1138390A24207D1A1490B22FDF7D2FC0EE0013421
S11383A00A2C0BDC2B1948335F780755002FF6D1C4
S11383B0351920210134E9710B2CF9D1984816267E
S11383C0066098483F21FEF79FF8002800D086E019
S11383D0934C17222260934F4521381CFEF794F8E2
S11383E0051E02D001357DD16EE17E6980239A009D
S11383F0291C301CFDF79BFC391C4931301C0B2215
S1138400FDF79EFC432763226620B4240821F17201
S1138410B075F4753276B2747776F774B073F4731A
S113842032747774804E7E4B356018251D607D4F05
S11384307D4C381C2B302168027891420FD2B868E9
S11384400918381CFEF760F8011E22D12668802224
S11384500136786992002660FDF769FC2AE1704DC7
S1138460002372491926236001242E600C706D4F7D
S11384700C2278696E49FDF763FC694A1A20106082
S1138480694D684E2968301C5F31FEF73DF8011EC6
S113849002D0013126D117E170690C22FDF747FCA7
S11384A02B685F4901331F242B600C605F48594AD5
S11384B0067815685C4F75433968A94209D3584951
S11384C0012E03D801360670192700E021270F601A
S11384D0F0E05F315348FEF717F8002806D001306A
S11384E000D1F1E04E4B32251D60C6E03B680133FC
S11384F0DCB23B60002C00D0DCE04E48FDF7FEFC13
S1138500D8E0484F43493B690E683A1C5F3B2B3225
S113851070001178181A01F093FA7D69464A6126B1
S1138520AE545221AE70F3264123444A6970297037
S11385307100F2266B54EB7071007223AB54013856
S11385406B54F4233E495A00060AF523A8546E548A
S1138550020C5E003B49F623AA55000E5E0003227E
S1138560AA556854F722384900205300374E6854FE
S1138570E8543749FF23A8555522AA205E006854C1
S1138580AA55381C4021FDF7BFFF00280BD1222536
S11385902560388B04210843388322484621FDF79F
S11385A0B3FF002805D0013000D18DE032212160D5
S11385B063E02848FDF7A2FC0F2727607AE0102724
S11385C03A425AD0244E174C3068216A884247D325
S11385D00D1C0A350A24A8420CD2441A0AE0316858
S11385E00CAD481E30602A1C0E48FDF7FBFF002826
S11385F003D0013C002CF2DA5CE0184A13682958D5
S113860004304F424F418021DB198F00B842F6D12C
S11386101360EEE768F9FF1F79BB000082BB00001E
S113862074FBFF1FD8F9FF1F78F9FF1F38FAFF1FEB
S1138630E7F0FF1F8EBB0000E7010000E50100002A
S1138640E9010000EB010000ED010000EF01000072
S1138650FF01000090BB000080F9FF1F80FBFF1F9B
S11386601B4EBA432A6035681A4F25630023F85617
S1138670BF21FDF75DFC00223A70079C0AA9033470
S1138680E07F0522FDF7AAF900281DD02B266E44B1
S11386903778002FF1D10BAA1278042AEDD10E48B5
S11386A0016813290BD10D4B01241E682425A64310
S11386B005601E604D200421FBF7E2FEDDE74D203E
S11386C0C821FBF713FFF5E78D2292009544F0BD16
S11386D080FBFF1F44FAFF1F74FBFF1F40FAFF1FBC
S11386E0F0B5071C08CF0E1C3A33197854225143B5
S11386F0864CA1B0651804952A30007800230390B5
S11387000593642504987968FDF750FF041E00D092
S1138710C1E00499387A4A694301D0180378002BE0
S113872003D00222E52B0BD105E0C07A040700D563
S1138730E8E00120E8E0039C144000D193E005E068
S11387400399114202D0642D00D195E0C17A3F24EF
S11387502A1C0C400F2C49D1002D47D05C060CD5A7
S1138760857F013DE9B2FD2904D8013A07AB9C1885
S113877000252570417B059103E0437B059CA342C2
S113878034D10D2A05DC07A80021FDF7D0FA002515
S11387902AE0847F6B461B339C54057F013B9D5428
S11387A0017E013B9954847D06AB9C54057D6C4647
S11387B01734A554817C013CA154037C013CA3548F
S11387C0857B05ACA554417A013CA154C379013C95
S11387D0A3544579013CA554C47804A98C54151CB0
S11387E040780D3D07AA5055EDB28BE0082319409F
S11387F000D087E0341C09340294027B231C944685
S1138800425C202A4AD1017A202908D01A1D2E243C
S11388101C70011C009201330A7A202A50D10021D5
S11388201970C37A3372C27F817F1406427F0B04AE
S1138830E41811026318047F1A193260417E047E21
S11388400B021A19B280C17D847D0B021A19F280C1
S11388500223642D44D0039C1C4006D1FDF762FC26
S11388600599884201D0642506E007AC6119029895
S1138870FDF7FDFB642501240498391CFEF7ADF8CF
S1138880C21D03D1012C3FD1102605E0002C00D1DC
S113889038E7002038E00426704235E0052A00D18C
S11388A0E5226446240705D5402A03D95A2A01D86B
S11388B02032D2B201311A7001330829A0D1A2E7C3
S11388C06446E40605D5402A03D95A2A01D8203241
S11388D0D2B2009C1A7001330131A3429CD19EE7AD
S11388E0039801241842C7D07E2171723219537A39
S11388F0002BC0D0202B01D82133537201340A2C11
S1138900F4D1B8E70024B7E721B0F0BDD8F9FF1FD0
S1138910F0B5ABB002900B7D00222B260C1C0D6829
S11389204A810596D80701D52E20059002992A314F
S11389300B70E281E789A289974200D33DE1029E50
S11389400C220436311C06A8FDF7FAF902980EA988
S1138950FFF7C6FE0490002803D0103001D00F2486
S113896010E0059863891F1868464130FDF78AFBBB
S113897022893918914207DD301C06A90C22FDF723
S1138980DFF90E24604219E16846868F1F27F3053C
S1138990720A37408A4E190F931903910193237D6C
S11389A0C68F012210A80178134200D180E0CB06C3
S11389B004D4114204D09223934003E0814B01E09C
S11389C0D22043000B2671198C466A1C642162452F
S11389D011D0501E9E0501D5017001E02D260670B0
S11389E07239C8B27221052801D87749095C5B0045
S11389F09BB20132EBE7281C74490A30FDF737FBC0
S1138A000EAD297A1023021C19400ED0029854236B
S1138A1006686F48311C3A310D785D4346191C369F
S1138A20F17BB0894843002100E00E98FDF792F8ED
S1138A3020220270451C039802380A2807D800F047
S1138A40EBFF090C0F1215181B1E21242700281CEC
S1138A5060491FE0281C60491CE0281C5F4919E09C
S1138A60281C5F4916E0281C5E4913E0281C5E4957
S1138A7010E0281C5D490DE0281C5D490AE0281C13
S1138A805C4907E0281C5C4904E0281C5B4901E0C0
S1138A905B49281CFDF7EBFA1221021C381CFDF778
S1138AA059F81021021C0198FDF754F8051C6DE0DB
S1138AB06B1C114201D0522200E02D222A700EAA12
S1138AC0157A591CAD0701D5482000E02D201870F7
S1138AD0157A4A1C6D0701D5532000E02D205870EB
S1138AE00EAB1D7A0132A80601D5412000E02D20ED
S1138AF04870381C1221FDF72DF82E27421C0770F0
S1138B0002210398FDF726F80021421C0770019802
S1138B10FDF720F8202202701221421CF00AFDF712
S1138B2019F876053A210170421C0221B00EFDF7B6
S1138B3011F80EAB051C187A102108420BD0277DC2
S1138B40F90704D4281C2F49FDF791FA051C238A40
S1138B50013323821AE009AE321C0E98FCF7FAFFA7
S1138B60301A1130071C2A1C013F03D32021117035
S1138B700132F9E7311C2818FDF779FA628A616835
S1138B800E9E01328B19051C6282636020276946A0
S1138B902F70681C4131FDF76AFA0A260D23037011
S1138BA04670851CE2892068049F291A013261817C
S1138BB0E281103700D0BDE6D1E600202BB0F0BD35
S1138BC0BC070000ED03000064B90000AFBB000067
S1138BD0D8F9FF1FBBBB0000BFBB0000C3BB000034
S1138BE0C7BB0000CBBB0000CFBB0000D3BB000061
S1138BF0D7BB0000DBBB0000DFBB0000E3BB000011
S1138C00E7BB0000EBBB0000F8B50D1C00243C27BB
S1138C1067430E4EF3191A8F002A12D11A1C3832E8
S1138C20012119879070002D05D0681880B2FBF7D8
S1138C3013FDB85100E0BD513C276743F019858608
S1138C4003E00134052CE2D10020F8BD48FAFF1FEF
S1138C5030B50D4C9622A544051C0C1C9200002135
S1138C606846FDF764F86846291C221C00F00EF8DB
S1138C70049B002B04D06846211C0022FDF70EFF44
S1138C80972189008D4430BDA4FDFFFFF7B5131C67
S1138C903A33051C1878141C542242430E1C8B4989
S1138CA08A18178B380600D409E100236B619E42B1
S1138CB000D184E0E08E009031782E2925D1777898
S1138CC02E2F22D12168002905D1278F4026374332
S1138CD027870E1C19E00098032800D8F1E0071C30
S1138CE0002B06D1009FC85D5C2806D02F2804D035
S1138CF0009F013FB8B20090F4E7B1780133002936
S1138D0001D1023603E00336D6E7002B57D0238F78
S1138D104021009F19432187A983032F3FD923684A
S1138D20D9190A7800270F700192208F10239843D5
S1138D3020872068211C0330FFF78AFF071E05D017
S1138D406E462468337900982354BAE031780029B8
S1138D5018D0A88BC0229043802318432087211C5D
S1138D60301CFFF775FF002802D0AF83071C09E011
S1138D70A98BC90506D52468009D711E6019FDF7ED
S1138D8076F91AE0AE8BF00503D56F463D88E5868B
S1138D9013E0684623680179009A995493E0D90551
S1138DA00DD5276803200025FD70211CE086201CBA
S1138DB0203008310C22FCF7C3FF052783E02E6026
S1138DC0208F434BA88303402387002E06D031789D
S1138DD0002903D00A2901D00D2901D1012010E076
S1138DE05C2901D02F290DD120273843A883767818
S1138DF0002E05D05C2E03D02F2E01D0022000E0DF
S1138E0004206861A98B0223261C194020360029FE
S1138E1025D15768101CEF602B3067610378D26846
S1138E205F43BF18A761271C1437201C21770C222D
S1138E30391C0830FCF784FF391C301C0C22FCF769
S1138E407FFF6B6908201843072121876861206828
S1138E50002804D01F49FDF70AF90322E286AF8BEC
S1138E60E4210F421CD0780602D5211C083111E000
S1138E70390613D46B690620211C034209D008313A
S1138E80301C0C22FCF75CFF6C690427BC4205D142
S1138E9019E01431301C0C22FCF752FF6E6006E01E
S1138EA0211C14316960301C0C22FCF749FF6A69EB
S1138EB005260027324206D10121296103E002215F
S1138EC000E003214F42381CFEBDC046D8F9FF1F05
S1138ED007FEFFFFFDBB0000F0B5041C031C87B0B8
S1138EE0171C626805913E3300201D78A087D007C7
S1138EF076D5A168E6688B1B01D1002089E09F42EA
S1138F0000D99FB2910305D5206C002802D1FDF74A
S1138F1019F92064542255433F494E19256C049590
S1138F20002FEAD0E3686946D805C20D03920C25E8
S1138F306B5A80208200D11A02938BB23D1C9F424F
S1138F4000D91D1C049AADB2002A0BD0301C211C80
S1138F500023FDF729FC00285BD1049B0398191812
S1138F60043110E0A16B049A2C4883185878002827
S1138F700ED05B68186C00280AD00368994207D1A8
S1138F8003994218111D05982A1CFCF7D9FE03E029
S1138F900832502AE8D126E0E168A28F68180599C2
S1138FA07F1BAB184D19E060A3870595318DBFB2C7
S1138FB000F08AFD0029B3D1A06BB2680130331CE4
S1138FC0A0632B33801A197800F07EFD0029A7D105
S1138FD0211C3431301CFDF7D7FC0028A0D018E048
S1138FE00924604215E0029A002A03D180208300FC
S1138FF09D4209D00095301C059A029BFDF720FC88
S11390000028C9D00424ECE7301C059AFDF7EAFADD
S1139010F6E707B0F0BDC046D8F9FF1F84F9FF1F7B
S113902038B50D1C096800290AD0FFF711FE041E8B
S113903008DB2968281D20310C22FCF781FE01E0A1
S113904011246442201C38BDF0B50B1C3E33071CB0
S1139050187854261F4C4643A5440C1C1E49102264
S11390608E19358B15402DD16068242318422BD0DE
S11390709622291C920004A8FCF759FE21680C22B0
S1139080203101A8FCF75CFE391C04A82268FFF714
S1139090FDFD089F002F19D02A1C04A82168FDF7A4
S11390A0FDFC821D12D1206801A90C2220300696F5
S11390B0FCF746FE211C8024049A04A82306FEF72C
S11390C02FFB03E0132100E00A2148429B26B6004F
S11390D0B544F0BD94FDFFFFD8F9FF1F426838B5D1
S11390E0041CD20605D500691B49C300CD18002213
S11390F06A70256C002D19D081208300E95C4A0731
S113910006D481229300E85C04218843E8540DE0EE
S1139110221C3E3213785420584310492A680818F8
S1139120291DFDF753F90130F2D0EAE76268002502
S113913093000AD5251C3E352B7854205843074903
S11391400918201CFEF77CFA051C201C002144226F
S1139150FCF7EDFD281C38BD84F9FF1FD8F9FF1F6B
S1139160F0B5824C031CA544059102923E33041CC5
S11391701878542646437E4900228E19A287358BDF
S1139180E90600D5E7E06768BA0700D4E5E0B9036B
S113919005D5236C002B02D1FCF7D4FF206406A86C
S11391A0256C04900299002900D1A7E0E368694680
S11391B0D805C70D03970C22505A0190002807D1F7
S11391C06C4F0299B94218D8A268D31A994214D2A2
S11391D0301C002D0AD0211C2A1C0023FDF7E4FAC0
S11391E0002800D0BDE0291D049119E0A16B06AA56
S11391F0FDF7F8F9002813D0B1E0002D0AD0301C97
S1139200211C2A1C0123FDF7CFFA002800D0A8E076
S1139210281D0490802704980021BA00FCF787FDDC
S113922080220398029F9300191A8F4202DD019F46
S1139230DA1B97B2049B0398059918183A1CFCF79B
S11392407FFD002D2FD081218B00EA5C0620024394
S1139250EA54A16B002329600193474A019811182D
S11392604B78002B0FD04A68106C00280BD029686B
S11392700368994207D1A84205D080220430291DF1
S11392809200FCF75DFD0198083001905028E4D16C
S11392900599E268CB19A168B8180593E060884283
S11392A009D9A06007E0301C0499A26BFDF78EF881
S11392B00130F8D0ECE7A38F0298FA18A287039A3A
S11392C0C11B2C488BB2D7190293874200DC69E793
S11392D0A16BB3680131321C2B32A163C81A117817
S11392E000F0F2FB0A1E00D05CE7211C3431301C74
S11392F0FEF764F9002800D154E732E0A28F002A77
S113930006D06568EA0305D58026B7053D43656048
S1139310002506E0201C311CFEF792F90028F7D046
S11393201FE0154B5E19707800280FD07168201C5F
S11393302C302C310822FCF777FE002806D1776800
S1139340A268F968BA608A4200D2FA600835502DE2
S1139350E7D1002005E0132402E00A2400E00424FD
S113936060428725AD00AD44F0BDC046E4FDFFFF7B
S1139370D8F9FF1FFF01000084F9FF1F70B5802397
S11393800A8F061C580010430887301C0C1CCD8E15
S1139390FFF75EFC0430092830D800F03DFB3A2F7B
S11393A0052F0A2F2F072931022433E00325E586F0
S11393B001362368002B23D03278002A11D0032DE4
S11393C002D95C21595501E0032D01D00135ADB21C
S11393D02368311C5819FCF74AFE2668821BE28672
S11393E00EE0E586022D00D103250020585507E044
S11393F0266803210025E186F57001E0032409E0D5
S1139400201C211C143020310C22FCF799FC002074
S113941001E00424604270BDF0B5031C3E33041C1B
S11394201878542646432D4D85B0AE19E368012AB9
S113943006D0022A12D0574257417D420D4012E015
S1139440002904DA4F4200259F420CD804E0A068AA
S1139450C51AA94200D9291CCD1804E0A268002528
S1139460914200D2551A9D4235D0271C34379D4273
S113947008D2211C2C31381C0822FCF761FC002383
S1139480E36003E0A1688D4200D90D1C328DE068D1
S1139490514208402940029201900391019B039A92
S11394A0934217D201990298B2680B187968019314
S11394B00131331C79602B33881A197800F004FBCE
S11394C00029EBD1301C391C0122FEF777F8002863
S11394D0E4D001E0E560002005B0F0BDD8F9FF1F3D
S11394E0F0B55F4C151CA54496220C1C920000217B
S11394F0071C02A8FCF71BFC22681C21138FA8067A
S113950000D40C210B43138702A8391CFFF7BEFBC0
S1139510061C0698002800D19DE08026F2012A400E
S1139520019204D06B46998C102001439984012345
S1139530EA0B1A4002A82168FDF7B0FA061E022EB3
S113954052D12168201C20310C221430FCF7F8FB86
S11395502168201C2C3108222C30FCF7F1FB2168F7
S1139560201C2C3108223430FCF7EAFB226801204D
S11395705368D97A014201D006218D436560D87FB2
S1139580997F000609044018597F1B7F090240187F
S1139590C1180020A160E0603A321278201C3E30ED
S11395A00270019013A91E380C22FCF7C9FB80231A
S11395B0990029400CD0019954220878294B424340
S11395C0201C99180222FEF79BFA0021A16007E0F3
S11395D0280505D5201C0222FFF71EFF002839D1DB
S11395E001206A0437D52FE06B0511D5B01D32D1A7
S11395F0276854223A373E781A4956436D00881931
S113960004906B0802A8211C029AFEF789F821E055
S1139610002820D12168201C20310C221430FCF7B2
S11396208FFB8022154365602568201C3A35297814
S11396303E300170201C203013A90C22FCF780FB63
S1139640019B002B07D0301C391C221C02ABFDF7F8
S1139650DFFC00E0061C301C9924A400A544F0BDE6
S11396609CFDFFFFD8F9FF1FF7B50C1C1D1C0A60F9
S1139670002A50D0131C3A331E7854214E43294FEC
S1139680BB191E8B10273E4202D026210D4244D125
S11396902F403AD000230193019E2349F700CF19AC
S11396A07E78002E2AD11023291C99430B1C211CDF
S11396B0FFF7DAFF022832D11B4A931958780028A1
S11396C00DD10836502EF7D1261C7C603F363378F6
S11396D002207B7065603D70019D256121E0596821
S11396E0201C2C302C310822FCF79EFC0028E8D1E9
S11396F00D498A5D1207E4D50B2411E0019B013367
S113970001930A2BC8D116240AE02764211C2A1CC1
S1139710FFF7E6FE05E00C2402E0132400E0062433
S11397206042FEBDD8F9FF1F84F9FF1FF0B50B1C82
S11397303A33071C18780D1C93B054264643019500
S11397402B8F27492022134301AC04228E192B8727
S1139750381C211CFFF7C4FE021E27D10CA806A941
S11397600822FCF7EDFA301CA169FCF71FFF002862
S11397702BD1237F72695801815C002908D0E52927
S113978025D1301C06A9FDF728F9C31DEBD120E033
S11397902B8F3020034304222B87381C211CFFF716
S11397A09FFE021E19D127687D6807E0022814D1A4
S11397B0276801227D68E87A02400CD1E5212970EE
S11397C0201C311CFEF79CF903E0042104E0012174
S11397D002E0021C01E00A214A42101C13B0F0BD51
S11397E0D8F9FF1FF0B50B1C3A33071C1878542620
S11397F046431A4C0D1C1A49A54496228E196846F4
S113980000219200FCF793FA348B10231C401FD1E3
S1139810288F082108432887391C68462A1C049489
S1139820FFF734FA049F002F14D06846291C221C29
S1139830FDF734F9831D03D000280BD1122508E06D
S1139840009A6846211C231C0296FDF769FF01E07B
S1139850132568429726B600B544F0BDA4FDFFFF6A
S1139860D8F9FF1FF8B5D30703D4164B1C68322C64
S113987025D154254543144E73191C8B10252540BE
S11398801BD1124F3D6040252C40082727430D4D26
S11398901F8314272F60550702D50D4A14431C83D8
S11398A05423584330180B224930FCF749FA4D2011
S11398B00421FAF7E5FD002003E0132000E0022074
S11398C04042F8BD74FBFF1FD8F9FF1F40FAFF1F89
S11398D0082000008268C36870B5041C9A4201D84D
S11398E000203EE04068820737D5211C3E310D78C8
S11398F054266E431B4A237F9619716958010D182B
S1139900301CA169FCF752FE002828D1E3681A0A2A
S1139910180C190EA3602B776A77A877E977632070
S113992043216623B422AB75EA752876A874697658
S1139930E974301CA169FCF7E7FD0130F9D0358BDF
S11399400123A06BB4689D433583A042C8D3483635
S113995031780222FCF790FE03E00A2600E0042698
S1139960704270BDD8F9FF1F38B5104B00241C5746
S1139970002C17D154250E4A684314600D4A1970FF
S11399801018056AC2690421A8180B4D0B4A013846
S1139990286015681020284310604D20FAF770FDE8
S11399A0201C01E01721484238BDC04644FAFF1F7D
S11399B080FBFF1FD8F9FF1F80F9FF1F40FAFF1F2C
S11399C010B5542460430B1C111C054A1018002BBD
S11399D002D1FCF7EBFD02E01A1CFCF703FE10BDFC
S11399E0D8F9FF1F70B5542670430D1C0549141C8B
S11399F00E18301C291C221CFCF7E8FC431CF8D070
S1139A0070BDC046D8F9FF1F5423584301490818B4
S1139A107047C046D8F9FF1F02B47146490849008F
S1139A20095C49008E4402BC7047C04603B47146C9
S1139A30490840004900095A49008E4403BC704754
S1139A40002934D00123002210B488422CD30124ED
S1139A502407A14204D2814202D209011B01F8E782
S1139A60E400A14204D2814202D249005B00F8E73B
S1139A70884201D3401A1A434C08A04202D3001B67
S1139A805C0822438C08A04202D3001B9C0822439A
S1139A90CC08A04202D3001BDC082243002803D0D8
S1139AA01B0901D00909E3E7101C10BC704700280A
S1139AB001D00020C04307B4024802A1401802901C
S1139AC003BDC046D90000000029F0D003B5FFF75C
S1139AD0B9FF0EBC4243891A1847C046002941D039
S1139AE010B4041C4C40A44601230022002900D5D4
S1139AF04942002800D5404288422CD3012424073F
S1139B00A14204D2814202D209011B01F8E7E40018
S1139B10A14204D2814202D249005B00F8E78842A4
S1139B2001D3401A1A434C08A04202D3001B5C081C
S1139B3022438C08A04202D3001B9C082243CC0879
S1139B40A04202D3001BDC082243002803D01B09D7
S1139B5001D00909E3E7101C6446002C00D54042FB
S1139B6010BC7047002806D003DB0020C043400827
S1139B7001E08020000607B4024802A140180290C8
S1139B8003BDC046190000000029EBD003B5FFF760
S1139B90A7FF0EBC4243891A1847C0467047C04607
S1139BA056312E342E3030340009022000010104D5
S1139BB0C000090400000208065005070501024020
S1139BC00000070582024000000A0343006F006E94
S1139BD000660055534243009C9C0000A09C00007A
S1139BE0029C00004C9C0000C99B0000819C00006A
S1139BF0800000000000000A0000000000000000D7
S1139C00000010034D0079002000500072006F0026
S1139C1064005553422052657365740A0D00555310
S1139C20422053757370656E6465640A0D00555364
S1139C304220526573756D650A0D00456E756D653C
S1139C407261746564202800290A0D0000008000F8
S1139C50011F000000755461736B657220555342F7
S1139C60746F53442D4361726420202020312E30C0
S1139C703003000000000000080001F800030002A7
S1139C8000080349006E0074000012011001000076
S1139C9000082504FC030001010203010403090474
S1139CA00A034D0061006E007500436C6F636B2006
S1139CB06C6F7373000820080045787465726E61D8
S1139CC06C00000030AC000033AC00000012000057
S1139CD043AC00004EAC0000051C00005EAC00006C
S1139CE06AAC0000051D00007DAC000086AC0000DD
S1139CF0050000009BAC0000A4AC000005010000BE
S1139D00BCAC0000C5AC000005020000D9AC0000EA
S1139D10E1AC000005030000FCAC000005AD000050
S1139D200504000025AD000034AD00000515000059
S1139D304FAD00005DAD0000051600007AAD0000D7
S1139D4086AD000005110000A0AD0000A5AD000027
S1139D500306000013AC0000FDAB0000000000008F
S1139D6018AC00001DAC000002000000310000002F
S1139D70312E35003200000057444F4700000000E8
S1139D8030AC000033AC00000012000018AC00003E
S1139D901DAC00000200000030AC000033AC000039
S1139DA00012000001AF000009AF0000070200002C
S1139DB025AF000030AF00000700000050AF0000E6
S1139DC058AF00000703000074AF000081AF00002B
S1139DD0070500007AAD0000ACAF000006020000E9
S1139DE0A0AD0000A5AD000003060000BFAF000059
S1139DF0C6AF000003070000DEAF0000E6AF0000BE
S1139E0003020000FFAF000005B0000001000000E5
S1139E1012B000001BB00000011A000013AC0000D7
S1139E20FDAB00000000000018AC00001DAC0000F9
S1139E300200000030AC000033AC0000001200004F
S1139E4042B0000027B000000404000040B000004D
S1139E5049B00000040B000063B000006BB00000C8
S1139E60010A00007FB0000086B00000010100007C
S1139E70A8B0000096B00000010D0000A4B00000DE
S1139E80AEB00000010E000013AC0000FDAB0000FA
S1139E900000000018AC00001DAC0000020000002F
S1139EA03F3F3F0074616D706572000030AC00008C
S1139EB033AC00000012000018AC00001DAC000020
S1139EC002000000556E646572766F6C746167659C
S1139ED000455A504F52540025AB000027AB0000F8
S1139EE0000400003FAB000041AB0000000500008F
S1139EF05CAB00005EAB0000000600006DAB000030
S1139F006FAB00000007000089AB00008BAB0000C2
S1139F100009000021A40000AAAB0000000A000010
S1139F202FA90000B9AB0000000E000031A9000009
S1139F30C8AB0000000F0000E5AB0000E7AB000079
S1139F4000100000FBAB000018AB00000011000083
S1139F5013AC0000FDAB00000000000018AC0000D2
S1139F601DAC000002000000536F667477617265D7
S1139F700000000030AC000033AC00000012000010
S1139F8085B10000C9B000000B0B0000F2B1000065
S1139F90D9B000000B000000F7B00000FCB00000D6
S1139FA00B17000022B1000027B100000B180000BD
S1139FB04FB1000055B100000B1900006BB1000057
S1139FC071B100000B1C00008AB100008DB10000CB
S1139FD00B010000DDB10000ACB100000B02000079
S1139FE0C2B10000C8B100000B040000E2B10000DF
S1139FF0E8B100000B03000002B20000F6B100005B
S113A0000B0C000009B200000FB200000B16000098
S113A0102BB2000031B200000B0500004BB200006F
S113A0204FB200000B07000095B200006AB20000B6
S113A0300B09000092B200009CB200000B0A000061
S113A040BDB20000C2B200000B080000DEB2000086
S113A050E4B200000B15000013AC0000FDAB0000DF
S113A0600000000018AC00001DAC0000020000005D
S113A0704C6F636B757000506F7765722D6F6E0057
S113A08030AC000033AC00000012000018AC00003B
S113A0901DAC00000200000030AC000033AC000036
S113A0A00012000018AC00001DAC0000020000000B
S113A0B057616B6575700033303000000000363036
S113A0C030000000003132303000000032343030D3
S113A0D000000034383030000000393630300000E1
S113A0E00031343430300000313932303000003344
S113A0F038343030000035373630300000313135F7
S113A10032303000323330343030000030AC0000B4
S113A11033AC00000012000013AC0000FDAB0000E3
S113A1200000000018AC00001DAC0000020000009C
S113A1304F444400004556454E004E4F4E4500578F
S113A140616B65757020726573657400486F737414
S113A150206465627567676572007065726970680E
S113A1606572616C206661696C757265000000003F
S113A17030AC000033AC000000120000C1AD0000A0
S113A180C4AD0000010F0000F1AD0000F4AD00000B
S113A1900110000020AE000023AE000001110000F9
S113A1A053AE00005BAE00000102000079AE000077
S113A1B081AE0000010B00009BAE0000A5AE0000C4
S113A1C001040000BCAE0000C7AE000001050000A1
S113A1D0A0AD0000E4AE0000010C000013AC0000D0
S113A1E0FDAB00000000000018AC00001DAC000036
S113A1F0020000004E4F4E45000000005254530030
S113A20000000000584F4E0000000000D89E0000DF
S113A2100F0C000075AA00000CA10000140300003C
S113A22084AA0000C49C0000160E000097AA000037
S113A23070A100000F0B0000A9AA0000989D000067
S113A240110D0000BCAA0000349E0000110900009A
S113A250CBAA000098A000000D020000DAAA0000BA
S113A26080A000000D020000E7AA0000749F000017
S113A2700D150000F4AA0000AC9E00000F020000BF
S113A28005AB0000809D00000F02000015AB00002C
S113A290536F6674776172652076657273696F6E49
S113A2A02000446576696365206964656E74696637
S113A2B069636174696F6E3A2000656E61626C65F2
S113A2C0640D0A0064697361626C65640D0A000AB6
S113A2D00A0D000A0D3D3D3D3D3D3D3D3D3D3D3DAD
S113A2E03D3D3D3D3D3D3D3D0A0D00206B427974B1
S113A2F0657300206279746573004E6F2053442D9A
S113A300436172642072656164790D0A00496E7656
S113A310616C6964206469726563746F72790D0A93
S113A320004469726563746F727920000D0A0A0033
S113A3305B445D002066696C6573207769746820EE
S113A340002062797465730D0A0020646972656384
S113A350746F726965732C200020667265650D0A3E
S113A3600046696C652F6469726563746F72792045
S113A3706E6F7420666F756E640D0A00777269746F
S113A38065206661696C6564004E65772066696C5A
S113A39065206C656E677468203D20000D0A524587
S113A3A04144204552524F52206F63637572656475
S113A3B00046696C65206E6F7420666F756E640D5F
S113A3C00A0052656164696E6720736563746F7215
S113A3D02000204641494C454421210D0A00577272
S113A3E06974696E6720736563746F7228732920BA
S113A3F00020536563746F722077726974652065F9
S113A40072726F72210A0D00202D204F4B0A0D002D
S113A410466F726D617474696E6720464154002DF5
S113A42031360031362000333220006E6F742070D4
S113A4306F737369626C650D0A00696E2070726FC8
S113A4406772657373202D20706C65617365207766
S113A4506169742E2E2E0D0A004D616B65206469AE
S113A46072206661696C65640D0A004372656174EB
S113A470652066696C65206661696C65640D0A0017
S113A4804E6577206E616D65206D697373696E67C3
S113A4900D0A004E6F7420666F756E640D0A0052CB
S113A4A0656E616D65206661696C65640D0A0044C2
S113A4B06972204E4F5420656D7074790D0A004402
S113A4C0656C657465206661696C65640D0A004697
S113A4D0696C65207375636365737366756C6C79F9
S113A4E0207472756E63617465640020636C7573A7
S113A4F074657273206672656564005472756E6368
S113A5006174696F6E206661696C65640D0A004947
S113A5106E76616C696420706174680D0A000D0ABE
S113A52053442D6361726420006E6F7420646574FB
S113A53065637465640D0A006E6F7420666F726DD6
S113A5406174746564002053444843002077726941
S113A55074652D70726F74656374656400427974F8
S113A56065732070657220736563746F723A00437B
S113A5706C75737465722073697A653A0044697204
S113A5806563746F727920626173653A0046415461
S113A5902073746172743A004641542073697A6579
S113A5A03A004E756D626572206F662046415473A1
S113A5B03A004C42413A00546F74616C20636C75EC
S113A5C073746572733A00496E666F2073656374C1
S113A5D03A004672656520636C7573746572733AEC
S113A5E0004E65787420667265653A004353443AB8
S113A5F000656E61626C650064697361626C65001C
S113A6000D0A496E76616C696420737769746368B6
S113A6100D0A000A0D415250207265736F6C766505
S113A620640A0D000A0D415250207265736F6C75F7
S113A63074696F6E206661696C65640A0D000A0DA9
S113A64053657269616C206E756D6265723A2000A3
S113A6504C617374207265736574206361757365EE
S113A660203D20000A0D53797374656D206D656D6E
S113A6706F7279207573653A0A0D0046726565201C
S113A68068656170203D20000A0D556E7573656420
S113A69020737461636B203D20005461736B20222E
S113A6A000222065786563757465642000207469F0
S113A6B06D6573202D20005461736B206475726185
S113A6C074696F6E205B6D696E2F61762F6D617892
S113A6D05D203D20002F00205B4D61782E206174A9
S113A6E02000205449434B735D202D2043505520B6
S113A6F03D2000250D0A00546F74616C20435055B1
S113A700207461736B206C6F6164203D20002520F0
S113A71028005461736B206D6F6E69746F72696E7B
S113A720672072657365740D0A000D0A546865200C
S113A73064657669636520686173206265656E206F
S113A7406F7065726174696E6720666F7220004273
S113A750616420706F7274206E756D6265720D0A8B
S113A760000D0A506F727420646972656374696FB6
S113A7706E3A20004F55545055540D0A00494E501E
S113A78055540D0A00496E76616C696420706F72CD
S113A790740D0A00506F727420697320696E7075AD
S113A7A0740D0A00506F72742073746174653A20DA
S113A7B000310D0A00300D0A000D0A3F3F0D0A2337
S113A7C0004D656D6F727920446973706C61790D09
S113A7D00A004D656D6F72792046696C6C0D0A0034
S113A7E04D656D6F72792057726974650D0A000AA0
S113A7F00D427965204279650A0D000A0D50617297
S113A800616D65746572207365740A0D000A0D54D8
S113A810656D702E20506172616D65746572207370
S113A82065740A0D000A0D506172616D657465727C
S113A8302076616C7565203D20000A0D4E6F2076F0
S113A840616C696420706172616D657465727320F6
S113A850617661696C61626C650A0D000A0D4F7264
S113A8606967696E616C20706172616D657465728F
S113A8707320726573746F7265640A0D000A0D4665
S113A8806163746F727920706172616D6574657251
S113A8907320726573746F7265640A0D000A0D503B
S113A8A06172616D657465727320696E76616C693D
S113A8B064617465640A0D000A0D4E657720506169
S113A8C072616D65746572732076616C696461741C
S113A8D065640A0D000A0D436F6E666967757261DF
S113A8E074696F6E2073617665640A0D00496E6346
S113A8F06F72726563742064617461206C656E6745
S113A90074680D0A000D0A53657269616C20636FE7
S113A9106E66696775726174696F6E0D0A004261D3
S113A9207564203D2000696E76616C69642100378E
S113A93000380020426974730D0A002073746F702C
S113A940206269742873290D0A00466C6F772063AE
S113A9506F6E74726F6C2000486967682077617449
S113A960657220004C6F7720776174657220005502
S113A9705342204572726F7220436F756E74657214
S113A980730D0A002D204352432D31362065727217
S113A9906F72733A002D204352432D352065727235
S113A9A06F7273203A00555342204572726F7220C1
S113A9B0436F756E746572732072657365740D0AE6
S113A9C0000D0A5365637572697479207365747434
S113A9D0696E67730D0A005465726D696E616C204F
S113A9E06D656E75206C6F67696E0054454C4E45FD
S113A9F054207365727665720020202054656C6E55
S113AA00657420706F7274206E756D626572203D7E
S113AA102000496E636F7272656374207365726996
S113AA20616C2073706565640D0A00496E636F7212
S113AA3072656374207061726974790D0A00496EDD
S113AA40636F72726563742073746F7020626974CB
S113AA50730D0A00496E636F727265637420666CCD
S113AA606F7720636F6E74726F6C0D0A000A0D0DA0
S113AA70004D41430020202020204D61696E206D4F
S113AA80656E7500204C414E20636F6E6669677574
S113AA90726174696F6E0020202053657269616C65
S113AAA020636F6E6669672E0020496E7075742F7F
S113AAB04F7574707574206D656E7500202020418B
S113AAC0646D696E2E206D656E75002020205374B0
S113AAD06174732E206D656E7500202020205553FF
S113AAE042206D656E750020202020493243206D80
S113AAF0656E750020204469736B20696E746572FD
S113AB00666163650020202046545020636F6D6D9C
S113AB10616E64730020202043414E20636F6D6D8D
S113AB20616E6473003100436F6E666967757265A8
S113AB30204C414E20696E74657266616365003213
S113AB4000436F6E6669677572652073657269612B
S113AB506C20696E74657266616365003300476FCB
S113AB6020746F20492F4F206D656E7500340047A7
S113AB706F20746F2061646D696E6973747261749F
S113AB80696F6E206D656E75003500476F20746FB8
S113AB90206F766572766965772F73746174697353
S113ABA074696373206D656E7500476F20746F2040
S113ABB0555342206D656E7500476F20746F2049B0
S113ABC03243206D656E7500476F20746F205344C7
S113ABD02D43617264206469736B20696E746572BD
S113ABE06661636500390046545020636C69656E84
S113ABF07420636F6D6D616E6473006100446973EA
S113AC00706C6179206D656E75207370656369661B
S113AC1069632068656C700071756974004C6561C6
S113AC20766520636F6D6D616E64206D6F64650081
S113AC30757000676F20746F206D61696E206D659B
S113AC406E75007573625F6572726F72730053681C
S113AC506F7720555342206572726F72730075735B
S113AC60625F636E745F72737400526573657420FF
S113AC7055534220636F756E746572730073657407
S113AC805F62617564005365742073657269616CF9
S113AC9020626175642072617465007365745F730A
S113ACA0746F70005365742073746F7020626974DC
S113ACB0732028312F312E352F3229007365745FAC
S113ACC062697473005365742064617461206269FD
S113ACD074732028372F3829007365745F7061728C
S113ACE00053657420706172697479202845564553
S113ACF04E2F4F44442F4E4F4E4529007365745FC9
S113AD00666C6F770053657420666C6F7720636F91
S113AD106E74726F6C2028584F4E2F5254532F4E1E
S113AD204F4E4529007365745F686967685F776192
S113AD307465720053657420666C6F772073746158
S113AD406C6C20282529205B312E2E39395D007347
S113AD5065745F6C6F775F776174657200536574B7
S113AD6020666C6F77207265737461727420282575
S113AD7029205B312E2E39395D0073686F775F634C
S113AD806F6E6669670053686F77207365726961D7
S113AD906C20636F6E66696775726174696F6E00AB
S113ADA073617665005361766520636F6E666967CB
S113ADB075726174696F6E20746F20464C415348FC
S113ADC0006D64004D656D6F727920446973706C19
S113ADD06179205B616464726573735D205B3C6CB4
S113ADE03E7C3C773E7C3C623E5D205B6E756D5DD7
S113ADF0006D6D004D656D6F7279204D6F646966ED
S113AE0079205B616464726573735D205B3C6C3EA6
S113AE107C3C773E7C3C623E5D205B76616C5D00F1
S113AE206D66004D656D6F72792046696C6C205BB0
S113AE30616464726573735D205B3C6C3E7C3C773B
S113AE403E7C3C623E5D205B76616C5D205B6E7592
S113AE506D5D007365745F64647200536574207083
S113AE606F72742074797065205B312E2E345D20EE
S113AE705B3C693E7C3C6F3E006765745F64647252
S113AE800047657420646174612064697265637449
S113AE90696F6E205B312E2E345D00726561645FD4
S113AEA0706F7274005265616420706F72742069EF
S113AEB06E707574205B312E2E345D007772697468
S113AEC0655F706F72740053657420706F727420C4
S113AED06F7574707574205B312E2E345D205B3079
S113AEE02F315D005361766520706F727420736535
S113AEF07474696E672061732064656661756C742F
S113AF00007365745F667470003C656E61626C65A5
S113AF102F64697361626C653E20465450207365EA
S113AF2072766572007365745F74656C6E65740027
S113AF303C656E61626C652F64697361626C653E29
S113AF402054656C6E657420736572766963650060
S113AF507365745F776562003C656E61626C652F32
S113AF6064697361626C653E205745422073657263
S113AF70766572007365745F7765625F6175746886
S113AF80003C656E61626C652F64697361626C6517
S113AF903E20574542207365727665722061757450
S113AFA068656E7469636174696F6E0053686F7766
S113AFB020636F6E66696775726174696F6E007283
S113AFC0656A656374005265736574206E6F6E2DD7
S113AFD07361766564206368616E6765730072658A
S113AFE073746F726500526573746F726520666165
S113AFF063746F72792073657474696E6773007219
S113B000657365740052657365742064657669635D
S113B01065006C6173745F72737400526573657458
S113B0202063617573650053686F772045746865A4
S113B030726E6574207374617469737469637300E8
S113B040725F69707374617400526573657420452E
S113B050746865726E65742073746174697374695D
S113B06063730075705F74696D650053686F772052
S113B0706F7065726174696E672074696D65006DC7
S113B080656D6F72790053686F77206D656D6F72AF
S113B09079207573650053686F77207461736B2032
S113B0A0757365007273745F7461736B73005265BA
S113B0B0736574207461736B20757365206D6561AD
S113B0C0737572656D656E740075744641542F63B3
S113B0D061726420696E666F005B706174685D20E4
S113B0E073686F77206469726563746F7279206323
S113B0F06F6E74656E740064697264005B70617471
S113B100685D2073686F772064656C65746564207E
S113B1106469726563746F727920636F6E74656EAF
S113B120740064697263005B706174685D207368A5
S113B1306F7720636F7272757074656420646972CE
S113B1406563746F727920636F6E74656E740069E1
S113B1506E666F66005B706174685D2073686F77FC
S113B1602066696C6520696E666F00696E666F643F
S113B170005B706174685D2073686F772064656C30
S113B1806574656420696E666F006364005B70615A
S113B19074685D206368616E6765206469722E203F
S113B1A0282E2E20666F7220757029005B706174E2
S113B1B0685D206E657720656D7074792066696CB2
S113B1C065007772697465005B706174685D2074F2
S113B1D065737420777269746520746F2066696C76
S113B1E065006D6B646972006E657720656D7074BF
S113B1F07920646972005B66726F6D5D205B746FA9
S113B2005D2072656E616D65007472756E630074A5
S113B21072756E6361746520746F205B6C656E6714
S113B22074685D205B706174685D007072696E742F
S113B230005B706174685D207072696E7420666969
S113B2406C6520636F6E74656E740064656C005B7E
S113B250706174685D2064656C6574652066696CF2
S113B26065206F72206469722E005B2D31365D207B
S113B2705B6C6162656C5D20666F726D6174202821
S113B280756E666F726D6174746564292064697388
S113B2906B0072652D666F726D6174005B2D3136C3
S113B2A05D205B6C6162656C5D207265666F726DBA
S113B2B06174206469736B2121212121007365630A
S113B2C074005B686578206E756D6265725D2064DC
S113B2D06973706C617920736563746F7200736550
S113B2E0637477005B686578206E6F2E5D205B70F9
S113B2F06174742E5D205B636E745D004A54414733
S113B300001000000000000000C0A80003FFFFFFC1
S113B31000C0A80001C0A80001A34831300000000B
S113B320C0B30000DAB300007E0400000700000090
S113B330CCB3000019B300000400000000010000B9
S113B34000000000000000000000000000000000F9
S113B35010007800200017005D000A000000004182
S113B360444D494E002020755461736B6572264B21
S113B370494E4554495300000000000000000000FD
S113B38000000000501403030000325F436F6E6E30
S113B390656374696F6E2074696D6564206F75747C
S113B3A00D0A000D0A0A48656C6C6F2C20776F72C9
S113B3B06C642E2E2E204B494E455449530D0A00E1
S113B3C066617669636F6E2E69636F003947656ED7
S113B3D065726174652E62696E00000001000100EF
S113B3E01010000001002000680400001600000096
S113B3F028000000100000002000000001002000D0
S113B4000000000000100000000000000000000028
S113B41000000000000000002165F25F2065F1EFEC
S113B4202065F2EF2165F22F00000000000000000B
S113B4300000000000000000000000000000000008
S113B44000000000000000000000000000000000F8
S113B45000000000000000002065F2CF2065F1FF2D
S113B4602165F2FF2065F2FF2065F1AF2166F20F3E
S113B47000000000000000000000000000000000C8
S113B48000000000000000000000000000000000B8
S113B4900000000000000000000000002165F24FE1
S113B4A02065F2EF2065F1FF2065F2CF2166F20FEF
S113B4B00CC1FF3F0000000000000000000000007D
S113B4C00000000000000000000000000000000078
S113B4D00000000000000000000000000000000068
S113B4E02165F20F2065F22F0CC2FF4F0BC1FFEF55
S113B4F00BC1FFFF0CC1FFEF0BC1FF2F00000000C9
S113B5000000000000000000000000000000000037
S113B5100000000000000000000000000000000027
S113B5202065F15F2065F1DF1693F85F0BC1FFCF53
S113B5300BC1FFFF0BC1FFFF0BC1FFFF0BC1FF9F3F
S113B54000000000000000000000000000000000F7
S113B5500000000000000000000000002165F29FD0
S113B5602065F1FF2065F1FF2065F1FF2165F2AF51
S113B5700FB2FC5F0BC1FFEF0BC1FFCF11AAFB3F62
S113B5802165F29F2065F25F0000000000000000CA
S113B59000000000000000000000000000000000A7
S113B5A02165F24F2165F2EF2065F1FF2065F1FF7F
S113B5B02065F1CF000000002165F21F2065F2FF35
S113B5C02065F1FF2065F1FF2065F1CF2165F22FA1
S113B5D00000000000000000000000000000000067
S113B5E000000000000000002165F29F2166F22F98
S113B5F00CC2FF5F0BC1FFEF0BC1FFEF1693F85FA7
S113B6002165F2CF2065F1FF2065F2FF2065F1FF8F
S113B6102065F22F00000000000000000000000080
S113B6200000000000000000000000000BC1FF0F3C
S113B6300BC1FFCF0BC1FFFF0BC1FFFF0CC1FFFF0D
S113B6400CC1FFAF1D72F36F2165F29F2165F20FEC
S113B65000000000000000000000000000000000E6
S113B66000000000000000000000000000000000D6
S113B670000000000CC1FF4F0CC1FFEF0BC1FFFF26
S113B6800BC1FFCF1693F81F2065F23F00000000A6
S113B69000000000000000000000000000000000A6
S113B6A00000000000000000000000000000000096
S113B6B000000000000000000CC1FF0F0CC1FF2FB0
S113B6C02065F28F2165F2FF2065F1FF2165F2EF1D
S113B6D02065F12F000000000000000000000000C1
S113B6E00000000000000000000000000000000056
S113B6F000000000000000000BC1FF5F0BC1FFEF62
S113B7001693F85F2065F1CF2065F1FF2065F2FF05
S113B7102065F1FF2065F1CF00000000000000006B
S113B7200000000000000000000000000000000015
S113B7302065F23F0CC2FF9F0BC1FFFF0BC1FFFF4F
S113B7400BC1FFFF0BC1FFAF1D74F45F2165F2EF66
S113B7502165F29F2165F20F000000000000000047
S113B76000000000000000002065F14F2165F2EFA9
S113B7702065F2FF2065F1CF0FB1FC5F0BC1FFEF35
S113B7800BC1FFFF0BC1FFFF0BC1FF9F00000000B7
S113B79000000000000000000000000000000000A5
S113B7A000000000000000002065F12F2065F1EF8B
S113B7B02065F1FF2065F1FF2065F1FF2165F29F0F
S113B7C00CC1FF9F0CC2FF2F00000000000000000E
S113B7D00000000000000000000000000000000065
S113B7E00000000000000000000000000000000055
S113B7F02165F25F2065F1FF2165F2CF2165F22F0B
S113B8000000000000000000000000000000000034
S113B81000000000000000000FFF000003FF000014
S113B82081FF0000C07F0000C03F0000800F0000C7
S113B830C1030000F0010000F8030000FE0700004F
S113B840FF010000FF000000FC000000F007000002
S113B850F00F0000FC3F0000436F6D6D616E6420CB
S113B8606C696E6520626C6F636B65640D0A000021
S113B870010000200000000013B90000054800008A
S113B880000000000400010018B90000D92D0000D8
S113B89045000200000000001CB90000817B00008C
S113B8A04500FFFF0000000023B90000A1140000C0
S113B8B02500FFFF000000002EB90000450600002F
S113B8C02500FFFF00000000000000000000000051
S113B8D0000000000000000011278913C509E304DB
S113B8E072023901D1009D004F0035001B000E008B
S113B8F048544D004A5047004749460043535300BB
S113B9004A530042494E00424D500049434F003FC4
S113B9103F3F0057646F6700617070004D6173733F
S113B9205374006D61696E74656E6163650075734F
S113B9306200015775616D4D4E73000000A0064012
S113B94000B0064000C006408913C509E304720232
S113B95039019D0069004F0028001B000E000700FC
S113B9600100000077727272727848000001AA87A1
S113B97053442D63617264206E6F7420726573701A
S113B9806F6E64696E670D0A0054494D454F5554F6
S113B9902121210D0A005772697465206572726F46
S113B9A0720D0A004552522D312121210D0A004603
S113B9B0696C653A20004469726563746F72793A00
S113B9C020002069732053464E0D0A00206973201D
S113B9D04C464E20000D0A5374617274696E6720E0
S113B9E0617420656E74727920002028636C75730D
S113B9F074657220004669727374206F626A6563AD
S113BA00742066726F6D20004669727374206F62D1
S113BA106A656374206572726F720D0A004C464E3B
S113BA20206F626A656374206572726F720D0A001A
S113BA3044617461203D00534E462046696C652084
S113BA406C6F636174656420617420656E747279CF
S113BA5020000D0A53464E206E616D652028007249
S113BA606561642D6F6E6C790068696464656E004D
S113BA7073797374656D00766F6C756D65204944D8
S113BA80006469726563746F7279006172636869D6
S113BA9076650029203D200020416C6961732043B4
S113BAA053203D20000D0A46696C65206C656E6765
S113BAB07468203D2000207374617274696E67207D
S113BAC0696E20736563746F7220002920464154A7
S113BAD020736563746F722000206F6666736574EB
S113BAE0200053442D6361726420766F6C74616727
S113BAF065206572726F720D0A0053442D63617282
S113BB0064205631206F72204D4D43202D206E6FDE
S113BB107420737570706F72746564210D0A00531C
S113BB20442D63617264205632202D2000486967D9
S113BB30682043617061636974790D0A00737461EC
S113BB406E646172640D0A004D616C666F726D659E
S113BB5064202D20004E4F542046415433322D2072
S113BB60004469736B2044206D6F756E74656400C6
S113BB704D53444F53352E30004641543332202028
S113BB8020004E4F204E414D4520202020002A0009
S113BB904469736B204420666F726D6174746564CC
S113BBA00D0A00554E44454C455445545854002004
S113BBB031203530322035303220004A616E004663
S113BBC06562004D617200417072004D6179004AF6
S113BBD0756E004A756C0041756700536570004FBF
S113BBE06374004E6F760044656300203C44495200
S113BBF03E202020202020202020202000443A5CC9
S113BC000040000000009549000000000069400069
S113BC10000000000100000000000000010100001D
S113BC20000210101010101010101010010101016A
S113BC3001000004040404040404040404040404CB
S113BC40040404040404040404040404042002207A
S113BC500000000808080808080808080808080878
S113BC600808080808080808080808080800200048
S110BC70007A0000000000770000000000D2
S113BC80555342530000000000000000005500001E
S113BC900400000004000000FF018021017001780D
S113BCA00906FCD57047FFF8FFFF0FFFFFFFFFFFFA
S106BCB0FFFF0F80
S9030410E8
